:020000040800F2
:100000002811002001010008F7370008D92800084E
:10001000F5370008410F0008E96300080000000000
:100020000000000000000000000000005D49000822
:10003000A71A000800000000613D00085D4C0008A0
:100040001B010008553B00081B0100081B010008AC
:100050001B0100081B0100081B0100081B01000810
:100060001B0100081B0100081B0100081B01000800
:100070001B0100081B010008611500081B01000896
:100080001B0100081B0100083D0700081B010008B8
:100090001B0100081B0100081B0100081B010008D0
:1000A000CD4C0008AD4D00081B0100081B010008E5
:1000B000B14D0008A1500008FD5200081B010008C6
:1000C0001B0100081B0100081B0100081B010008A0
:1000D0001B010008E15E00081B0100081B0100086D
:1000E0001B0100081B0100081B010008DFF80CD0F1
:1000F00000F0E6FA00480047E974000828110020E3
:100100000648804706480047FEE7FEE7FEE7FEE7B1
:10011000FEE7FEE7FEE7FEE7FEE7FEE77D4C0008B0
:10012000ED0000082DE9F0410024061B254671F181
:10013000000605DA01240027D0EB070067EB010178
:10014000161E73F1000605DA0027D2EB070201251F
:1001500067EB030300F0D0F986460E4617469C462F
:10016000AC4204D00025D0EB050E65EB010624B1AE
:100170000020D2EB000760EB030C704631463A4694
:100180006346BDE8F08140EA01039B0703D009E024
:1001900008C9121F08C0042AFAD203E011F8013B73
:1001A00000F8013B521EF9D2704780EA010210B5F7
:1001B00002F00043400022D04A001FD0010E01EBA4
:1001C0001261C0F35600C2F3560240F4000042F43C
:1001D0000002A0FB022000047F39140400D0401C60
:1001E00050EA124001D44000491EC2B20C0604EB92
:1001F000D010401C4008802A02D003E0002010BD2F
:1002000020F00100002900DA0020184310BD2DE97C
:10021000FE4F81EA030404F0004421F00041009401
:100220004FF0000B23F0004350EA01045ED052EA85
:1002300003045BD0C3F30A54C1F30A552C44A4F25F
:10024000F3340194A0FB0254C1F3130141F4801173
:10025000C3F3130343F4801301FB024400FB034E7A
:10026000840A970A44EA815447EA8357A4FB076843
:1002700002958D0A05FB07854FEA932C04FB0C546D
:100280002705029D4FEA065847EA1637B5EB0805E1
:100290006EEB070C870E920E47EA811742EA831233
:1002A000A7FB0201B6EB0B0164EB00042B0D43EA44
:1002B0000C335E1844EB1C50DA465146E7FB020152
:1002C000C5F313044FEA0B3343EA14534FEA0432E5
:1002D000019C43EA0603A4F10C040294009CCDE9BE
:1002E00000B400F09FF903B0BDE8F08F0020014694
:1002F000F9E72DE9F04D81EA030404F0004B21F009
:10030000004514464FF0000A23F0004150EA050270
:1003100020D054EA01021DD0C5F30A570246C5F3A6
:100320001303C1F31300C1F30A5640F4801543F4DC
:100330008013A7EB0608101BD64608F2FD3873EBB6
:10034000050002D308F1010801E092185B41B8F101
:10035000000F03DA00200146BDE8F08D00204FF4C5
:100360008011064684460EE0171B73EB050705D384
:10037000121B63EB050306434CEA010C49084FEAE4
:10038000300092185B4150EA0107EDD152EA0300B8
:1003900012D082EA040083EA0501084305D0101B4D
:1003A000AB4106D20122002306E000224FF00043B9
:1003B00002E06FF0010253101AEB06004CEB0851FB
:1003C00010EB0A0041EB0B01BDE8F04D00F01BB94A
:1003D00070B521F0004303430CD0C1F30A5500244B
:1003E000D5EB040564EB0403D617AD1AB34102DB69
:1003F0000020014670BD201841EB025170BDC10FB5
:1004000080EAE0700844CA079623002100F0CDB8C6
:1004100096230022114600F0C8B80EB5C10F80EA3D
:10042000E0700844CA07002140F233438DE80E0013
:100430000A460B4600F0F6F803B000BD0EB540F2D8
:10044000334102910021CDE900110A460B4600F02C
:10045000E9F803B000BD00F0004220F00040C10DFB
:10046000C0F3160040F400007F2901DA0020704735
:10047000962903DCC1F19601C84001E09639884015
:10048000002AF4D04042704770B5C1F30A5201F01F
:1004900000450024C1F3130140F2FF3341F4801101
:1004A0009A4201DA002070BD40F233439A42A2F230
:1004B000334203DC524200F05FF800E090402C43EE
:1004C000F1D0404270BDC1F30A5210B5C1F313011F
:1004D00040F2FF3341F480119A4201DA002010BD4E
:1004E00040F233439A42A2F2334203DC524200F01C
:1004F00043F810BD904010BD2DE9F05F0546002087
:1005000092469B4688460646814640241BE0284684
:1005100041464746224600F02FF853465A46C01A35
:10052000914110D311461846224600F016F82D1AB4
:1005300067EB01084F4622460120002100F00DF82C
:1005400017EB00094E41201EA4F10104DFDC4846F0
:1005500031462A464346BDE8F09F202A04DB203A74
:1005600000FA02F1002070479140C2F1200320FA06
:1005700003F3194390407047202A04DB203A21FA04
:1005800002F00021704721FA02F3D040C2F12002AC
:1005900091400843194670470029A8BF7047401C86
:1005A000490008BF20F00100704710B4B0FA80FC89
:1005B00000FA0CF050EA010404BF10BC704749B1C6
:1005C000CCF1200421FA04F411FA0CF118BF012136
:1005D00021430843A3EB0C01CB1D4FEA00614FEA16
:1005E000102042BF002010BC704700EBC3501044E5
:1005F0000029A4BF10BC7047401C490008BF20F070
:10060000010010BC704710B5141E73F1000408DA25
:10061000401C41F1000192185B411A4301D120F0C6
:10062000010010BD2DE9F04D92469B4611B1B1FA83
:1006300081F202E0B0FA80F220329046FFF78DFF9F
:1006400004460F4640EA0A0041EA0B0153465A4667
:10065000084313D0114653EA010019D0C8F14002F3
:100660005046FFF789FF05460E465046594642461A
:10067000FFF773FF084305D0012004E02046394608
:10068000BDE8F08D0020054346EAE0762C43374371
:100690000A986305E40AA0EB08000022FD0A44EA78
:1006A00047540A3002D500200146E9E70105101938
:1006B0006941DDE9084500196941BDE8F04DA2E74F
:1006C000064C074D06E0E06840F0010394E807009F
:1006D00098471034AC42F6D3FFF70CFDE0980008C1
:1006E0000099000870B58C1810F8015B15F007032D
:1006F00001D110F8013B2A1106D110F8012B03E0BB
:1007000010F8016B01F8016B5B1EF9D12B0705D4C2
:100710000023521E0DD401F8013BFAE710F8013B0B
:10072000CB1A921C03E013F8015B01F8015B521E27
:10073000F9D5A142D8D3002070BD000070B54F4C50
:100740004FF490652946204600F01BFA002866D039
:100750002946204600F0A8F849490888401C08802E
:100760000121204600F0ECFA464942F21072B1F83D
:100770005000904202D2401CA1F8500007F09CF8B3
:1007800005F094F9404DB5F91410B5F9120005F0D3
:100790005DFF3E4CA5F856002080A16820468847A2
:1007A000A088A5F8580003F08FF807F081F9384EBB
:1007B000384C3078082833D045F6AC30606042F6CB
:1007C000EF60A06042F2C400E0603348008A2080FD
:1007D000208E6080A16B2F488847208E69882F4C1F
:1007E00008444FF6FF7101EA80006887207A4FF0D5
:1007F000000540071DD501F0E5FA294949F6A24058
:100800000880284840F21A62C188491C89B2C18018
:10081000914204D3A16821F00401A160C58070BD9C
:1008200041F2130060604FF48060A06040F61B50FE
:10083000CAE730780A281BD2DFE800F01A0616054E
:100840000A050D1A1114EAE7BDE8704006F0A2B8D7
:1008500008F028F908E0BDE8704002F07FBD06F01E
:100860001FFC01E007F07CFABDE8704007F078BAA1
:1008700000F0FEFB84F8B65070BD0000002401407B
:1008800024070020480100206400002040070020C9
:100890001B070020E4000020F8010020A402002033
:1008A000442C0140600900206FEA1121016070476B
:1008B0000029816802D041F0010101E021F001012D
:1008C000816070470029816802D041F4807101E0A5
:1008D00021F48071816070472DE9F041824E92B021
:1008E000304600F00BF90BA800F039FA01214FF463
:1008F000C06003F0EBFA00248DF831404FF4602023
:10090000CDE90D044FF4A0204FF009080B9001270A
:100910008DF83C808DF830700BA9304600F080F9DE
:10092000724D8DF831408DF830708DF83C700BA908
:10093000284600F075F901231A460F21304600F0D1
:10094000C0F9022201231146304600F0BAF9012312
:1009500003220021304600F0B4F901230422194695
:10096000304600F0AEF9012305220B21304600F09D
:10097000A8F9012306220421304600F0A2F9012340
:1009800007220821304600F09CF9012308220321A8
:10099000304600F096F9012309220A21304600F082
:1009A00090F90121304600F084F90121284600F039
:1009B00080F901231A460521304600F055F901233C
:1009C0001A460621284600F04FF90021304600F073
:1009D000CBF84FF4E041284600F0C6F8012130463C
:1009E00000F0B8F80121284600F0B4F801213046A3
:1009F00000F0A6F80121284600F0A2F801213046B7
:100A000000F09EF90121284600F09AF940F61451B1
:100A1000374804F04AFF12208DF8400002208DF87C
:100A200041008DF842408DF8437010A802F010FF8D
:100A300001224FF49061304600F0E8F80121304681
:100A4000FFF740FF01213046FFF732FF0121284622
:100A5000FFF72EFF304600F06EF9304600F09FF8A9
:100A60000028FAD1304600F075F9304600F082F8DF
:100A70000028FAD1284600F05EF9284600F08FF8E9
:100A80000028FAD1284600F065F9284600F072F8EF
:100A90000028FAD10121084603F0F4F9154D284643
:100AA00000F09AFD684600F042FE0F4801A94C3064
:100AB0000090114881E811018020CDE904404000F8
:100AC000069080000790202008904FF44050CDE918
:100AD00009046946284600F00DFE0121284600F071
:100AE0006FFD12B0BDE8F0810024014000280140F4
:100AF000002C014008000240B40200200D4910B54E
:100B0000884202D1012144150AE00B49884202D1F2
:100B10000121041504E0094988420AD10121CC03CE
:100B2000204603F0DFF92046BDE81040002103F025
:100B3000D9B910BD0024014000280140003C01400B
:100B40000029816802D041F4801101E021F4801174
:100B5000816070470029816802D041F4004101E0C2
:100B600021F4004181607047826822F4E0420A4328
:100B700082607047014600208968490700D501203E
:100B8000704710B50246002054680B0AC9B20C40E9
:100B90001168194202D0002C00D0012010BD01467E
:100BA00000208968090700D50120704738B5012168
:100BB0001C2003F08BF9FF20ADF8000000248DF815
:100BC000034003258DF8025069460D4801F0F4FA00
:100BD0000120ADF800008DF803408DF80250694601
:100BE000084801F0E9FA2320ADF800008DF8034031
:100BF0008DF802506946044801F0DEFA38BD000065
:100C000000080140000C014000100140002A426829
:100C1000C9B201D00A4300E08A4342607047000035
:100C200010B542680E4B0C791A400B6842EA042258
:100C30001343436083680B4A1340D1E902422243C5
:100C40004C7943EA44031A438260C26A097C22F465
:100C50007002491EC9B242EA0151C16210BD0000D2
:100C6000FFFEF0FFFDF7F1FF70B5072409290AD94F
:100C7000C568A1F10A0606EB4606B440A543B34099
:100C80001D43C56007E0056901EB4106B440A5437B
:100C9000B3401D430561836BC3F30154121B921CC7
:100CA00002EB82041F22A2409343A1400B438363C3
:100CB00070BD826B491E22F4401242EA01518163E9
:100CC000704770B5072409290AD9C568A1F10A0639
:100CD00006EB4606B440A543B3401D43C56007E09C
:100CE000056901EB4106B440A543B3401D430561CE
:100CF0001F23072A09D2446B521E02EB8202934043
:100D00009C4391400C43446370BD0D2A09D2046B8F
:100D1000D21F02EB820293409C4391400C43046338
:100D200070BDC46A0D3A02EB820293409C4391402D
:100D30000C43C46270BD816841F008018160704756
:100D40000029816802D041F4A00101E021F4A00152
:100D500081607047816841F0040181607047002123
:100D60000160017141718160C160012101747047AE
:100D700070B51E4C214694F83800B1F84250062850
:100D80001ED9B4F84A10B4F84C00A1EB000202F1ED
:100D90000902122A04D8FFF751FB0022144B0AE083
:100DA000884204D2FFF74AFB0022124B03E0FFF710
:100DB00045FB0022104BFFF72AFAFFF784FB09E0FE
:100DC00005D12846FFF73AFB0C4A0D4BF3E70D49D6
:100DD00051F82000C5EB45116063B0EB410F03D91A
:100DE000C5EB45104000606370BD0000500400205A
:100DF00000003440000033400000354067666666FE
:100E000066E64B40908F000810B50C4C20784007E8
:100E100013D5FFF7ADFF0A49A08E08800848303887
:100E2000018821F010010180001F018841F01001AC
:100E30000180207820F00400207010BD50040020B4
:100E400040040040F0B4184816494FF49677436CBC
:100E500008468A68046815485FEAC25C42F00806E2
:100E6000007822F008054FEA047415D5002C08DB41
:100E7000120714D408B1082811D1BB420FDA8E60D2
:100E800007E012070BD508B1082808D1BB4206DAE3
:100E90008D60F0BC05F006BF002CF2DAE8E7F0BC8C
:100EA00070470000A4020020480100201B0700201A
:100EB00070B506464089204B204C4FF480710025C8
:100EC00080B362887AB1012A0CD1E188491C89B2C9
:100ED000E1803289914205D36580E580FF2801D009
:100EE000401E708170BD70882288904201D9012215
:100EF00000E00022184601F0E8F97088B18801444A
:100F00002088401C80B220808142EBD82580A088B8
:100F1000401C80B2A080F1888842E3D30120608029
:100F2000A58070BDFFE70022184601F0CEF9A5802C
:100F3000E58025806580F4E7000C0140C0050020B5
:100F4000FEE70000FCB505464FF6FF7600200C4694
:100F5000ADF8006048F205078DF8040020E000BFFE
:100F600015F8010B8DF8040001A9084602F0D3F82A
:100F7000BDF800009DF8041080EA0120ADF80000E3
:100F80005FF00000BDF800100A0402D587EA4101B5
:100F900001E006EA4101401CADF800100828F1DB31
:100FA000641EDDD26946084602F09FF8BDF80000D5
:100FB000FCBD00000246002004E000BF12F8013B27
:100FC0001844C0B2491EF9D27047000070B5144AE7
:100FD00085B010880024134901940094039420469E
:100FE0000494138807E00D8B009E35440095CD8B4B
:100FF000019E3544019515889D42F4D0401CC0B235
:101000008028EED3009841110748418084800198E0
:101010004111064881830183818205B070BD0000C3
:1010200024070020A4020020DA050020C8040020C4
:1010300030B50E4902880A800C4A4388083A13806A
:101040000B1F808818802024151F2C800020401C36
:1010500080B27328FBD341F21110088044F6480097
:10106000108047F2480018802C8030BD202C0140B1
:10107000114944F648000880091D46F648000880DA
:10108000091D41F2111008800B48001F018841F032
:101090002001018009480021A0F86410A0F8621026
:1010A000A0F86010A0F85E10A0F85C10A0F85A102C
:1010B0000348418181827047182C0140A40200201E
:1010C000640000202DE9F04F544B55480021DA7A96
:1010D00090F800C0802A2CF001067DD31C68514B8B
:1010E00002F01F0253F822204F4B14421A6802D01C
:1010F00042F0200201E022F0200299461A604A4B99
:10110000DFF828B1DFF828A193F84650494B9BF847
:101110000040B3F90430022C6ED1B9F80840C4F392
:10112000C007C4F30024A74266D03F4C2C3C94F87F
:101130000280B8F1000F09D0394FB8F1010FB7F9AB
:1011400002700DD0B8F1020F1AD127E0110558D561
:10115000910656D40121A1702CF00401017050E0D9
:1011600016054ED496064CD55FEA4C7607D44CF063
:101170000406067037B1418026F00101017002219A
:10118000A1703EE04380002BF9DD46F001010170C3
:101190002949CE6A4661896A8161F0E7B0F806C0E4
:1011A000BCF1000F01D1002B19DC90F80CC0AC454C
:1011B00015D107F26667BB4211DC204FBF895FEA99
:1011C000477C0CD45FEA877C09D45FEA427C06D571
:1011D0005FEA826C03D500E01CE0FF0711D00670C7
:1011E0004180AAF80010418141618161A17089F8B4
:1011F0000F108BF8001004E006704180AAF8001070
:101200004181C3800573500960F3CB22C9F80020E7
:10121000BDE8F08F067041804181F9E7E0050020CC
:1012200044090020F0930008A40200201B070020BE
:1012300024010020DA05002064000020540A002068
:101240002DE9F04796B000240C940D940E940F9461
:1012500072B69048816941F400718161816941F4FD
:10126000806181614FF4004002F002FE8A4D00214E
:101270002846FFF727FB00212846FFF719FB874E7A
:1012800000213046FFF714FB854F0021384600F05F
:1012900097F901204FF47041401C8842FCD3284646
:1012A000FFF72CFCB1463046FFF728FC384600F02B
:1012B00093F94FF46020CDE912048DF845400120E8
:1012C0004FF004088DF8440010948DF8508010A958
:1012D0002846FFF7A5FC01231A4605212846FFF7FB
:1012E000F0FC0123022206212846FFF7EAFC012335
:1012F000032207212846FFF7E4FC012304220F21E3
:101300002846FFF7DEFC384600F066F9684600F034
:101310000EFA6148634E4C300090CDF80C80CDE958
:1013200001648020CDE904404000069080000790D1
:10133000202008904FF44050CDE909046946384612
:1013400000F0D8F901212846FFF7BCFA0121384600
:1013500000F036F901212846FFF7AAFA47F230518A
:1013600015941598401C15908842FAD301212846FF
:10137000FFF7E6FCADF82C40A04640F2DC5A4FF4F3
:10138000007420E05046CDF854801599491C159101
:101390008142FAD330880D9908440D9070880E99D7
:1013A00008440E90B0880F9908440F90F0880C996B
:1013B00008440C9001212846FFF7C2FCBDF82C0020
:1013C000401CADF82C00BDF82C00A042DAD30D98DB
:1013D000354A40F3CF1633480A3006830E9941F35D
:1013E000CF1444830F9941F3CF1383830C9941F3B6
:1013F000CF1CA0F804C0ACF5C05C40F2C371ACF5E2
:101400009B7C8C450ED2A6F5C856363E8E4209D23C
:10141000A4F5C854363C8C4204D2A3F5C853363BDD
:101420008B4203D3D18841F48041D180D1884904D3
:1014300007D41E49028B21F85C2F428B4A80808B97
:10144000888000212846FFF73DFA0021384600F049
:10145000B7F800212846FFF72BFA00214C464846F2
:10146000FFF726FA0220C102401C8842FCD328461E
:10147000FFF744FB2046FFF741FB384600F0ACF88D
:10148000FFF72AFA0A493C20087062B616B0BDE898
:10149000F0870000001002400024014000280140B5
:1014A0000800024026050020540A0020B40C002049
:1014B00018070020F0B5284B40F22D4643F6FB25D7
:1014C0005C6C264BB4F5FA5F13DDB4F5FA4F10DC13
:1014D00041F6AD17A4F5FA54674306EBA7364FF46F
:1014E000B5777C4305EBA41475106410C3E904546C
:1014F00001E0C3E904651D69D5605C69401A546167
:1015000010609168884202DA4942884200DC11602A
:1015100010684443107E0441906A21189162506A19
:10152000814200DD9062916A106A814201DB0846C7
:1015300000E09062986111684D43117C0D410841B3
:101540002918B2F91C00884204DBB2F91A0088425B
:1015500000DC08B2F0BD0000480100202801002096
:1015600010B54FF40054204600F0ACF8002813D01A
:101570000A49087840F008000870204600F014F886
:101580000021074800F01CF80648C17E012903D15C
:101590000021C1760121017710BD00007A060020EC
:1015A00044000240580B0020C10002D502490860E7
:1015B000704702494860704704040240000002403E
:1015C0000029016802D041F0010102E04FF6FE72ED
:1015D000114001607047000001684FF6FE72114033
:1015E00001600021016041608160C1603149314A80
:1015F0000839904203D1486840F00F0006E02D4AB8
:101600001432904204D1486840F0F00048607047BE
:10161000284A2832904203D1486840F47060F5E7C8
:10162000244A3C32904203D1486840F47040EDE7D0
:10163000204A5032904203D1486840F47020E5E7D8
:101640001C4A6432904203D1486840F47000DDE7E0
:10165000184A7832904203D1486840F07060D5E76C
:10166000154A111F904203D1086840F00F0006E0B0
:10167000114A1432904204D1086840F0F00008602A
:1016800070470D4A2832904203D1086840F47060D8
:10169000F5E7094A3C32904203D1086840F47040B3
:1016A000EDE7054A50329042EAD1086840F47020D4
:1016B000E5E700000800024008040240406880B2EC
:1016C0007047000001460020CA0001D5034A00E02F
:1016D000034A12680A4200D0012070470004024009
:1016E00000000240002A026801D00A4300E08A4359
:1016F0000260704730B5036847F6F07293430C6A96
:101700008A682243D1E904452C4322438C69224351
:10171000CC6922434C6A22438C6A22431A430260FA
:10172000CA6842600A6882604968C16030BD0021B1
:10173000016041608160C160016141618161C1619D
:10174000016241628162704710B5114C8CB000217A
:101750002046FFF735FF2046FFF73EFF0D4800907B
:101760000D480021CDE901016420CDE9030180206D
:10177000CDE905010791089109910A916946204632
:10178000FFF7B8FF01212046FFF71AFF0CB010BD8C
:101790005800024004380140B007002010B5012174
:1017A0008CB0084602F06EFB1E4C00212046FFF76D
:1017B00007FF2046FFF710FF1B4800901B480190D1
:1017C00000211020CDE902018020CDE9041006910E
:1017D0000791089109910A9169462046FFF78AFF0F
:1017E000012202212046FFF77DFF01218DF82F10F5
:1017F00004208DF82D008DF82E100E208DF82C0071
:101800000BA802F025F80F208DF82C000BA802F091
:101810001FF801212046FFF7D3FEFFF795FF0CB01C
:1018200010BD000044000240043801404C07002075
:1018300030B540F6AA21204AC184838B1488E31A6C
:101840009BB20F2B10D312888283037E002253B1E8
:101850001A4BB3F90A30062B05DB194B1B78022B08
:1018600003D0002B00D1828430BD164B40F68B256F
:101870005B6CA3F22D14AC420FD2428B521C92B27D
:101880004283642AF0D364224283B0F924208A423E
:1018900001DA02EB2111818430BD41F29414A3429C
:1018A000FADBB0F92430002B02DDA3EB211100E0BC
:1018B00000218184428330BD240700206400002081
:1018C0001B0700204801002010B50446B0F90200B3
:1018D00043F6991148438113E06840F26662504331
:1018E00001EBA030E060B4F9001043F699125143C7
:1018F0008A13216940F26663594302EBA1312161E9
:1019000004F044FE6061A18840F6AB220844401018
:10191000A0F515415539E062914205D9A0F5F8517D
:10192000FF39521C91421DD249F25451884202DDC6
:10193000A0F5204002E0A0F5F850FF38206300EB4E
:10194000400040F34F002085B4F924104A429042F1
:1019500001DA104602E0884200DD0846E083228476
:1019600061848AE0A0F5FE42FF3A41F255518A4275
:1019700014D8A2F6AA20206300EB400040F34F00E9
:101980002085B4F924205142E183884201DA0846D7
:1019900002E0904200DD1046404250E0A0F5D44203
:1019A000AA3A8A4215D2A2F6AA20206300EB400090
:1019B00040F34F012185B4F924004242E2832084A0
:1019C000914201DA104602E0814200DC0846608460
:1019D00053E0A0F5AA42543A41F256539A4215D226
:1019E000A2F6AB20206300EB400040F34F002085BF
:1019F000B4F924104A42904201DA104602E08842CB
:101A000000DD08464042E083218419E0A0F58042D1
:101A100041F254539A4215D2A2F6AA20206300EB59
:101A2000400040F34F012185B4F92400E083424295
:101A3000914201DA104602E0814200DC084620842F
:101A400062841AE0A0F52852AB3A8A4215D2A2F677
:101A5000AA20206300EB400040F34F012185B4F938
:101A60002400E08342422284914201DA104602E0DF
:101A7000814200DC08464042A9E7B4F91E00A0EB11
:101A800040208013E080B4F92000A0EB40208013B8
:101A90002081B4F92200A0EB40208013608110BDAA
:101AA00001210176704770471548164A4FF480416E
:101AB0000078042821D002F13C03D08A9B88C01A08
:101AC00000B22F2801DD001108E0002801DD002010
:101AD00007E00D4B984201DA184602E0402800DD8D
:101AE00040209389184400B2884203DC40F26661CA
:101AF000884200DA08469081704791817047000063
:101B00001B070020C8040020C0FEFFFF38B54B486B
:101B10004B4902880B889A1A92B20F2A71D309880E
:101B2000484C01804FF0FF01E2884FF47A7355046E
:101B30004FF4967002D51622009103E0950403D568
:101B400015220091014670E0D50402D514220091BF
:101B5000F8E7150502D513220091F3E7550502D5E4
:101B600012220091EEE7950502D511220091E9E7D6
:101B7000D50502D510220091E4E7150602D50F2203
:101B80000091DFE7550602D50E220091DAE79506AF
:101B900002D50D220091D5E7D50602D50C22009181
:101BA000D0E7150702D50B220091CBE7550702D5E8
:101BB0000A220091C6E7950702D509220091C1E7E4
:101BC000D20702D008220091BCE72289550702D52E
:101BD00007220091B6E7950702D506220091B1E7EA
:101BE000D20702D005220091ACE7A27AD20702D038
:101BF00004220091A6E7A289D40603D5032200910E
:101C0000A0E719E0140702D5022200919AE75407D1
:101C100003D4940701D4D20702D00122009191E7A6
:101C20000020034602460146009002F043FFBDE853
:101C300038400248FFF73CB938BD0000480A002090
:101C400024070020540A0020F0B5594859498288D9
:101C50000B889A1A92B29C2A64D3098881805649CB
:101C60000A880146002A0B7843F0020156D1164635
:101C7000524A1C0715680246127822F0020274D5F7
:101C80004F4C0746E4887F785FEA845C02D547F0D2
:101C9000010701E027F001074770A704477802D544
:101CA00047F0020701E027F002074770670401D4FC
:101CB000E70703D0477847F008074770640603D565
:101CC000447844F0040404E01C0603D4447824F06F
:101CD00004044470EC0450D4354C9A07247824F062
:101CE000100423D4324D42782F7A2D78012A45F002
:101CF000100514D0022A16D02D4C042AA47804F121
:101D0000010C0CF0FF0C13D0072A25D0032A23D096
:101D1000052A21D0062A1FD021F0100142E0B90780
:101D200002E00570F0BD39070029FADB0470F0BD50
:101D3000FA0601D41A060AD50170022C04D280F8E2
:101D400002C0BCF1020FF2D341F080012AE021F081
:101D5000100101708670F0BD877A7F06F7D5032CDD
:101D600004D8017080F802C0F0BD0FE05107D8D54B
:101D70001906D6D443F0800114E002704178CB07F5
:101D800001D18907F0D522F010010BE0E9040BD452
:101D90009907E9D4818AC82902D2491C8182E3E7E4
:101DA00043F00A010170DFE702708682DCE7000081
:101DB000FC0600202407002026070020A4020020A3
:101DC000540A0020094944F648000880091D46F6D7
:101DD00048000880091D41F6CC4008800348001FD8
:101DE000018841F02001018070470000182C01405B
:101DF000084946F668000880091D0880091D41F25F
:101E0000555008800348001F018841F020010180DF
:101E100070470000182C014010B5C28800210AB19B
:101E2000032206E002890AB1022202E0428912B1CD
:101E30000122027000E0017004784FF4804344F600
:101E4000206244B1012C06D0022C07D0032C01D112
:101E50004180818010BD4380828010BD41F23331CA
:101E6000418040F6B731F4E730B5B1F86A5000234D
:101E70001A240D22854202DCB1F9680030BD4D887C
:101E8000854202DBB1F9000030BD01EB82056D88AF
:101E9000854201DD144601E013DA134604EB030228
:101EA0004FEA52029A42F0D101EB830231F823103B
:101EB00054889288521A001B424301EB622000B200
:101EC00030BD31F9220030BD054920B1086940F02C
:101ED00080000861704703484860034848607047C5
:101EE0000020024023016745AB89EFCD06494FF43E
:101EF0007A70CA68D20705D0401E0004000CF8D1E1
:101F0000FF20704700207047002002400E4A032047
:101F1000A2F1500182F83E00002048810B4908865A
:101F2000C862C8830884488490620948816CB1F50E
:101F3000206F01DBA3219162807A002802D0906A91
:101F4000404290627047000064000020300500208D
:101F5000480100200449002048810881C862886245
:101F6000024988627047000064000020C008002019
:101F7000F0B53B4988894A89801A80B20F2866D318
:101F800088894881CA8937480B3A272A26D28A7815
:101F900022BB8268364B42F480728260324A354CF2
:101FA000354D12785607314A0AD4344E3688168099
:101FB000334A12881A80334A12882280324A09E052
:101FC000324E36881680324A12881A80314A128878
:101FD0002280314A12882A8001228A702F4B304D8C
:101FE00019469A7F0968802A32D302F01F0255F8F9
:101FF000222011422CD0826822F48012184E826076
:10200000123614461215B778521C62F38617254A09
:10201000B77093F816C01778BCF1800F27F002064E
:1020200008D30CF01F0C55F82CC011EA0C0F01D18D
:1020300047F0020616701A7E802A0DD302F01F02A6
:1020400055F82220114207D144F400218160F0BDEF
:10205000826842F48012D1E724F40021F6E7000000
:1020600018070020A402002048010020C00400201E
:10207000C2040020C4040020C6040020B0040020D4
:10208000B2040020B4040020B6040020B8040020EC
:10209000BA040020BC040020BE040020E00500209B
:1020A000F0930008C804002070B520488189028997
:1020B000891A89B20F292FD3818901811C4B1D48B0
:1020C00019465D7A06681C4C096846F00402802DAA
:1020D00007D305F01F0554F82550294201D126F0F9
:1020E000040202609A7B802A17D302F01F0254F880
:1020F0002220114211D1026822F002020260DA7A33
:10210000802A0ED302F01F0254F82220114208D177
:10211000016821F00801016070BD026842F002020E
:10212000ECE7016841F00801F5E70000180700201E
:10213000E0050020A4020020F0930008F0B51D4C3B
:102140001B4A4FF0010C94F83B5094F80AE01446F7
:1021500092F83C3094F838402B43651CEEB2154D94
:1021600095F83D700025BEF1FF0F0AD0BEF1000FBB
:1021700006D18B4213D155700C2C01D282F83860F5
:10218000F0BD834202D182F801C0F5E78B42F7D15E
:102190005570B80709E000BF82F83850F0BD83429F
:1021A000FCD1F84382F801C080070028F4D0F0BDCC
:1021B0005004002048010020F0B5CA78002502F044
:1021C0000F03D20601D58A7813430A784FF00F0E19
:1021D00012F0FF0F4FF001021CD004680F8802FAC2
:1021E00005F63740B74211D14FEA850C0EFA0CF7CD
:1021F00024EA070703FA0CF43C43CF78282F02D0D7
:10220000482F02D002E0466100E006616D1C082DF7
:10221000E4D304600C88FF2C1ED944685FF00006EC
:1022200006F1080702FA07F50F882F40AF420FD1D9
:102230004FEA860C0EFA0CF7BC4303FA0CF73C434A
:10224000CF78282F00D14561CF78482F00D1056184
:10225000761C082EE4D34460F0BD0000F0B5144CA9
:10226000002801DAE36900E06368420D120185B2DB
:10227000C0F301579540C0F30346032F05D0C202B7
:102280000AD50322B240934307E023F070626368EB
:1022900023F07063636002E0AB4343F0706201B10E
:1022A0002A43002801DAE261F0BD6260F0BD00005F
:1022B000000001400246002092680A4200D001203E
:1022C000704741617047016170470AB10161704711
:1022D000416170470F4A104B92F838105B5C8342A3
:1022E00001D1012004E00D4B5B5C834203D100204F
:1022F00082F83A0070470A4B5B5C834201D181202F
:10230000F6E7084B595C814201D18020F0E70320B9
:10231000EEE7000048010020A8980008BA980008DD
:10232000AE980008C09800080A4810B501784FF030
:1023300000024C0708494FF0FF0389684FEA01711A
:1023400005D5002901DA827210BD837210BD002903
:10235000FBDBF8E748010020A4020020F0B5194E8D
:10236000194C0022E31CA6F1060CB75CA518ED7809
:10237000FF5C0D430F43BD421FD01CF80270FF5C91
:102380000F43BD4219D015460023A618F6780E4318
:10239000C6545B1C1CF80220DBB2062BF5D3C178B7
:1023A00081700179C17000214218491C15711CF817
:1023B0000550C9B20629F7D3F0BD521CD2B2032A88
:1023C000D3D3F0BD828F00085004002010B5024620
:1023D0000021064B06205C186478944200D1084620
:1023E000491CC9B20629F6D310BD000048010020DF
:1023F000214810B590F8671000222048012936D1F5
:102400001F49898899BB1F491E4B4C6C40F6B83157
:10241000B3F86E308C4227DD1B49097821BB90F858
:102420002711491CC9B280F82711C8291CD380F88C
:1024300027210146D0F82C4191F82811A34203DD51
:10244000052908D2491C01E041B1491E80F8281134
:10245000C9B2052902D3012180F82611191B074CA6
:102460002C3C6162C0F82C31B3F5FA6F03D280F8CE
:10247000262180F8282110BDB40C0020A4020020E1
:10248000DA050020480100201B0700204FF4C0425D
:10249000C260002181620E22028241F26202426128
:1024A000082202834FF46042428381834FF07842D6
:1024B000C0E9082140F6C41101807047B0F900104E
:1024C000B0F90220891A41604269037E4A431A41E9
:1024D000836A13448362426A934200DD8262836AA4
:1024E000026A934200DA8262C268836A4A43017CCC
:1024F0000A410B41D118B0F91C208A4201DA10467A
:102500007047B0F91A008842FADC08B27047000040
:1025100010B514481449B0F88C200B889A1A92B25E
:10252000B2F5437F1DD90988A0F88C10B0F88A1045
:1025300020F8581F002242860C480D4CC288828029
:10254000C180C38983812489891AA4B2C48181602E
:10255000E11A0161074A818AC182928A8282511AF4
:10256000816110BD48010020240700207C0C002060
:10257000300500206400002009480A49B0F8AA206C
:102580000B889A1A92B241F684639A4206D309885C
:1025900020F8AA1F418881800021418070470000F7
:1025A00048010020240700200D480178C90702D007
:1025B0000C49098801E04FF6FA71C165094901200B
:1025C0001039088007482438018841F00101018052
:1025D00004481838018821F0180101807047000074
:1025E00048010020240400400A49D1F8902012B18B
:1025F000521EC1F8902031F88A2F521C21F81A2956
:102600004A6A521C4A628A8F521C8A8701F8380C27
:1026100070470000480100201CB52D4890F83B3061
:1026200090F83C20934252D000248DF8044053404F
:102630008DF800309DF800300122012B08D09DF864
:102640000030022B09D09DF80030042B0AD00DE099
:102650001F498DF80420443108E01D498DF80420FD
:10266000463103E01A498DF8042048319DF80420D2
:10267000012A2CD190F83D309DF80040154AA34224
:1026800017D090F83E309DF80040234208D0B0F8B3
:102690004C30A0F84A300B881488E31AA0F84C306C
:1026A00090F838302BB1B0F840301488E31AA0F815
:1026B000423012880A80A0F8402010F83E1F9DF892
:1026C0000020114300F801199DF8001001701CBD95
:1026D000500400202407002070B5344D40212846C6
:1026E000FFF7E8FD840080212846FFF7E3FD44EA78
:1026F0004004A9152846FFF7DDFD0443E1B22C4C48
:1027000094F870508D4250D04D4084F87010012DD7
:1027100003D0022D01D0042D47D194F87400A843B2
:1027200084F8740094F87320AA420FD084F8735090
:1027300094F8722001238B401A4207D11A4384F87F
:10274000722094F87110491C84F8711094F871107B
:10275000042928D330B1012811D002280FD0042831
:102760000DD012E01348C18821F04001C1802078CB
:10277000002184F83B1020F06000207005E02178F3
:1027800041F02001217084F83B000B4994F83B0094
:1027900091F82720904204D081F827000749202093
:1027A000087000F00DF884F84C5070BD0010014026
:1027B00048010020540A0020B40C00201807002013
:1027C00070B50D4D40212846FFF774FD840080212F
:1027D0002846FFF76FFD44EA4004A9152846FFF795
:1027E00069FD04430548072100F8704F017100217D
:1027F00041708170C17070BD00100140480100201F
:1028000070B5344890F83A10CA43920761D001F08D
:10281000030280F8392090F83D305B061B0E80F8EB
:102820003D30012A01D0812A02D15B1C80F83D3065
:102830000278D2074DD0DBB203F00102C3F34004AB
:10284000A24246D1B0F84E400025641CA0F84E408C
:10285000204CA0F8505090F83E60A47AB24202D0CA
:1028600080F83E200DE0A607B6EB837F02D080F80B
:102870003F5006E090F83F30642B02D25B1C80F89A
:102880003F3090F84030642B0CD25B1CDBB280F8F8
:102890004030022B06D204F00103934202D10222FF
:1028A00080F84020012901D0002912D190F8382069
:1028B000C16D00EB820291610163D0E906121144FF
:1028C000D0E908231A441144826A1144C26A1144AF
:1028D000416370BD48010020FEE700002DE9F04F84
:1028E00000BF00209E4E9F4AA6F51271A6F5BE7944
:1028F000A6F1440B06F1440E804601F5E074A1F107
:10290000780301F5457A1D5C15F0C00706D0402F0D
:1029100051D0C02F77D0802F76D004E115F01F055D
:1029200004D0154440F080072F7201E082F808803F
:10293000012826D0022824D0032822D0042820D021
:1029400008281ED010281CD0874D55F820C0DCF870
:10295000005054F820703D40CCF80050824D55F89E
:1029600020C0DCF8005056F820703D43CCF80050F1
:102970001D5CAD0659F820502F6813D53AF810C0E9
:102980003EE051F820502F6854F820C007EA0C07A9
:102990002F6051F820502F6856F820C047EA0C07E6
:1029A0002F60E5E7DFF8B8C10CF1F00C5CF820C04F
:1029B00007EA0C077EE015F01F0504D0154440F02F
:1029C00080072F7201E082F8088001281DD00228BC
:1029D0001BD0032819D0042817D0082815D0102898
:1029E00013D0614D55F820502F6854F820C007EAE5
:1029F0000C072F605C4D55F820502F685BF820C005
:102A000047EA0C0756E00BE056E051F820502F68DB
:102A100054F820C007EA0C072F6051F82050ECE76B
:102A200015F01F0505D0154440F0800785F821708A
:102A300001E082F82180012825D0022823D0032834
:102A400021D004281FD008281DD010281BD0464DA7
:102A500055F820C0DCF8005054F820703D40CCF808
:102A60000050414D55F820C0DCF800505EF8207051
:102A70003D43CCF800501D5CAD0615D53A4D3AF8F3
:102A80001070CC3514E051F820502F6854F820C055
:102A900007EA0C072F6051F820502F685EF820C01D
:102AA00047EA0C072F60E6E72D4D3AF81070E03D3D
:102AB00055F820502F6036E015F01F0505D015445D
:102AC00040F0800785F8217001E082F8218001281C
:102AD00030D002282ED003282CD004282AD0082851
:102AE00028D0102826D0204D55F820C0DCF8005002
:102AF00054F820703D40CCF800501B4D55F820C0D4
:102B0000DCF80050164F883757F820703D43CCF85A
:102B100000501D5CAD06B1D4114F3AF81050E03FA3
:102B200057F820703D60401CC0B21128FFF4EBAE96
:102B3000BDE8F08F51F820502F6854F820C007EA04
:102B40000C072F6051F820502F68DFF814C00CF1EB
:102B5000880C5CF820C047EA0C072F60D9E700001A
:102B60007C960008E0050020789400084FF4077177
:102B7000C1824FF45861018340F61451818370473C
:102B8000F0B5C48AB0F900608681B0F90250C58101
:102B9000B0F904300227002101220382AB4204DB9A
:102BA000B54202DDC78042810CE0B34204DBAE4295
:102BB00002DDC78041811CE09D4205DBB34203DD9D
:102BC000C2804781018115E0B54204DB9E4202DDEF
:102BD000C280418105E0AE4205DB9D4203DDC1803C
:102BE0004281078106E09E4204DBAB4202DDC180E8
:102BF00047810281C388458900EB430700EB450507
:102C0000BB89AE899B1B0FFA83FEA0F812E00689F0
:102C1000AB8900EB460CBCF80CC0A3EB0C03838221
:102C2000B0F91830B7F90CC0A3EB0C0CB4EB4C0F97
:102C300004DA80F82010A3F1A10113E0A64503DD1A
:102C400080F82010B9890BE026B1012E04D0022EA5
:102C500010D004E0062100E0052180F82010A989A9
:102C6000091B6D31418309B2B1F5586F04DB5B1E5E
:102C7000438304E00421F0E7002900DC4283418B18
:102C80008183F0BD0B49002288760A62CA614A62DC
:102C9000094A32F9103002EB40028B62B2F902208D
:102CA000CA62064A32F810000882A1F86000A1F852
:102CB00062007047F8010020D2980008C69800080A
:102CC0002DE9F05FF748F84982880B889A1A92B28A
:102CD0000F2A44D30988F54A81808146118801244E
:102CE000F348F44E002579B3491E1180C573F24BA9
:102CF00085620168B3F902304F0742F6AA2218D460
:102D0000F78847F40057F780EB4E3678B60709D5B9
:102D1000866826F080068660A0F87C5080F87E5099
:102D200080F87F50CE0404D480F8F040C0F8EC5016
:102D300003E080F8F0504E0707D4934205DB80F89B
:102D4000F440A0F8F25004E010E080F8F4504E0790
:102D500003D4934201DBC90703D080F81151BDE8C9
:102D6000F09F80F81141A0F81251F8E78046B0F8C2
:102D7000181143F69820814202D2491CA8F8181174
:102D800001F0AEFECD4FDFF81CB397F85000ABF169
:102D90001C0B10B1FEF796F905E09BF8001021F02E
:102DA00001018BF80010FFF723FB00F0CBF9C448BA
:102DB00041F26801426C4FF400608A4201DBC14974
:102DC00004E0B2F57A6F02DABE49091D086097F88F
:102DD0005100DFF8DCA2BC4BBC4FC007AAF12C0AA3
:102DE0003AD0987B802833D398F8001089072FD4E5
:102DF00098F80F008AF80500AF48514690F800C0D7
:102E00002CF0020C80F800C0ABF80250CBF8145044
:102E10009BF800C02CF0010C8BF800C0B079400684
:102E200011D44889B0F5FA7F03D2401CAAF80A00F1
:102E300012E040F63C70824201DD002007E10820EC
:102E40008AF8034003E1CD700020AAF80A50FEE0A2
:102E50008AF80350AAF80A50D8F80800010501D5ED
:102E60000820F4E0954991F83FE05FEACE7149D03F
:102E7000954B98F80F208AF805205B7A4146802B05
:102E80004CD30B785B0735D4F3889B0405D500BF82
:102E900020F02000C8F8080034E0ABF80250CBF86E
:102EA00014509BF800C0884B2CF0010C8BF800C02C
:102EB00040F020008860D87D80280AD300F07F0C85
:102EC0001B684FF0004020FA0CF0034201D10C7156
:102ED00000E00D710879C00702D15FEA8E7005D558
:102EE0000320032A01D08AF80840B0E00020C8F887
:102EF0002850ACE020F02000C8F80800F08820F44A
:102F00000050F08098F82601444601280BD06B4809
:102F100090F8630048B1FDF795FF0FE00A6842F0B2
:102F200004020A60B4E7092091E0A068C10502D557
:102F300020F0080001E040F00800A06094F846206E
:102F40004FF48041E2B143F69913012A1FD0881E45
:102F5000032A3A78C2F3810220D0012A23D0022A20
:102F600021D0A4F814115A4890F85E00042812D019
:102F7000A4F84410514890F87000012816D025E0BC
:102F800043F21E50A4F8140143F2333008E042F635
:102F9000CC42A4F81421A4F84430EBE7A4F81401BF
:102FA000A4F84400E6E7A4F81401DCE7387842F21C
:102FB0006662C0F3810001280FD0022810D041F6CC
:102FC000E12000BFA4F81401A4F844209BF80020DD
:102FD000D20708D0BBF8022007E0A4F81421F3E7D9
:102FE0004FF40050EEE734488288A9F8122010B25E
:102FF000B4F944205043C0F38F325046AAF812204F
:103000008A4200D9418233490978C90605D5428AE6
:1030100041F233318A4200D241822189C1F3C00298
:10302000C1F300218A4205D1428A40F6CC418A424E
:1030300000D94182B17AC90700D04582BAF812009E
:10304000A06200287FF7F9AE23480570022099F8A6
:103050001A1099B9022841D080B119490B789C0601
:1030600008D5B479640605D51A4C2478E40964F3CC
:1030700086130B70F18821F40A61F1801049496CC4
:103080004E290ADBF1880B0607D521F08001F1807B
:1030900009490B7823F002030B7089F81A0088F8AD
:1030A0000F005CE6600900202407002026070020AE
:1030B000A4020020540A0020DA050020B40C0020ED
:1030C00048010020100C0140E0050020C804002049
:1030D00064000020FC06002038070020398F0029FA
:1030E000BBD143F698213987B7E770B500230C8828
:1030F00063F30F02012505FA03F6344206D0C3F14B
:103100000F0605FA06F1114361F30F025B1C102B49
:10311000F1DB028070BD70B500230C7863F3070209
:10312000012505FA03F6344206D0C3F1070605FA75
:1031300006F1114361F307025B1C082BF1DB0270FF
:1031400070BD0000F0B51F4890F866301E48012B96
:10315000816821F4006232D11C4BDE8874062ED4C3
:103160001B4D0F054FF00004B5F902501ED4194A4B
:10317000526C642A11DC40F6386295420DDAB204D2
:103180000BD4027852070ED4B0F8D42040F6B835EC
:10319000AA4203D2521CA0F8D420F0BD41F4006131
:1031A00081605C81F0BDA0F8D440F0BD41F2CD015A
:1031B0008D42FADD997AC907F7D18260F3E7826020
:1031C000F0BD0000B40C0020A4020020540A00202E
:1031D000DA05002048010020F0B5364D364F044690
:1031E00095F83B0097F83B1023780843EE1C627873
:1031F000834205D1E0781146FEF7A0FF207908E070
:1032000094F802C084450CD1E1781046FEF796FF91
:10321000E07905F82F0F2878805D6870287BE877C3
:10322000F0BD82421DD161461846FEF787FF95F832
:103230004E1095F83B00814207D1B97A09B1A179C6
:1032400000E0617985F82F101EE06978012901D02E
:10325000A17922E0617927E0297841F00401297001
:1032600012E0E1788142DBD119466046FEF766FF45
:1032700095F84E1095F83B0081420AD1B97A09B110
:10328000617ADFE7217ADDE715F82F1F895D697024
:10329000C5E76978012906D0617A85F82F10B97AD7
:1032A0000029F1D1D8E7217A85F82F10B97A0029C1
:1032B000EAD0D1E750040020480100200B480178F3
:1032C00021F0020100F8381B002100F8181941779D
:1032D000817733218185418508214184012100F8CE
:1032E0001F1C034880F8391070470000500400206C
:1032F000480100200D4900B50B4851F8012F40F856
:10330000032F89888180084801210930FFF726F8BA
:10331000054802211330FFF721F8034804211D302E
:103320005DF804EBFFF71AB85004002048010020B4
:10333000094944F648000880091D46F648000880FF
:10334000091D41F2111008800348001F018841F057
:103350002001018070470000182C01402DE9F04742
:10336000664C674B0025A0780126654A1033052876
:103370007ED2DFE800F00313113E1100108820F028
:10338000010010801D805F480580001F0580001F20
:103390000580FFF7CDFFA670BDE8F087594941F2DF
:1033A00044401C390880574945F6580024390880A4
:1033B000091D47F25800088052492020283908800A
:1033C0000020401CC0B27328FBD3FFF7B1FF4C496B
:1033D00084F85C502C3147F69060088048481430DF
:1033E00006801D80108840F0010010800220A0702F
:1033F000D2E700215FF0010004EB410204EB40033F
:10340000B2F85020B3F850309A4200D20146401C26
:10341000C0B20628F0D33C48405C84F83900FFF77E
:103420004DFF1D2000F0F3F900F076F8374E3848D4
:103430004FF4807996F83B10012904D002291BD063
:10344000042930D047E040218046FEF733FF870053
:1034500080214046FEF72EFF47EA40074946404696
:10346000FEF728FF074347F0010084F83B0000E027
:103470003DE0224809302CE040218046FEF71AFF4B
:10348000870080214046FEF715FF47EA400749467E
:103490004046FEF70FFF074347F0020084F83B0069
:1034A0001648133015E040218046FEF703FF8700E1
:1034B00080214046FEF7FEFE47EA40074946404667
:1034C000FEF7F8FE074347F0040084F83B000B4882
:1034D0001D3002F045FF94F82F0086F838001D20BB
:1034E00000F0ABF90420A0700A48057054E710887A
:1034F00020F0010010801D80A5704DE750040020D1
:10350000000800403C2C0140888F00084801002042
:10351000001001401B0700202DE9F041344C14F845
:103520002F0F344DE07240212846FEF7C3FE86007F
:1035300080212846FEF7BEFE46EA4006AF15394612
:103540002846FEF7B7FE0643207BF1B22F3C8142AE
:1035500015D084F83C0040212846FEF7ABFE8600DB
:1035600080212846FEF7A6FE46EA40063946284650
:10357000FEF7A0FE064384F83B60FFF74DF81E4DB2
:1035800095F83B00012827D0022828D0042829D00C
:10359000174894F83B102730085C04F8300F14F8F3
:1035A0000109FEF713FF04F82F09A87A00B10120E2
:1035B000607001F02DFB94F84E0094F83B108842A7
:1035C00006D094F83800062802D2401C84F838004F
:1035D00084F84E10BDE8F0810548093004E0044845
:1035E000133001E002481D30BDE8F041FFF7F4BDA3
:1035F0005004002000100140480100202DE9F04156
:10360000524991F87200AA287ED191F8730055288A
:103610007AD14F4C00200A5C2254401CC0B274285E
:10362000F9D34C4E2069C6F80100A08AA6F805001F
:10363000D4F81600F060D4F81A003061D4F81E00F7
:103640001234706102F032FE4349608A888102F0D0
:1036500047FE207D123CC007307802D040F00400C5
:1036600001E020F004003D4930704FF480403C4DB3
:10367000886114F8280F85F82000608B6880A08B83
:10368000A880E08BE880208C2881608C354F688191
:1036900094F8240087F8D20014F8011C304686F80C
:1036A0003B100026C0F89460FFF724FE2E48A18E40
:1036B0000183E18E4183218F818394F84210283C5D
:1036C000012908D0022901D0032909D0297821F045
:1036D0000C01083107E0297821F00C01091D02E0F6
:1036E000297841F00C01297094F86E20012162B113
:1036F000012A01D0022A0BD087F8461094F86430D2
:103700001A4A4BB1518108E014E087F84660F5E7AA
:10371000022287F84620F1E7568194F870100129BB
:103720000AD094F86D1051B101290BD04FF480519B
:10373000A0F87610BDE8F08144F21C71F8E74FF470
:103740000051F5E741F25551F2E7000000FC000896
:10375000B40C002048010020640000204C0C002024
:10376000C8040020A402002030050020540A0020D4
:103770007CB50121082000F0A9FB4FF48070ADF862
:10378000040010248DF8074001208DF8060001A9DF
:103790001548FEF711FD0121092000F097FB0121DA
:1037A0001248FEF75BFD0820ADF8000004208DF8FC
:1037B00003000F4E03258DF8025069463046FEF790
:1037C000FBFC08213046FEF77CFDADF800408DF88B
:1037D00003408DF8025069463046FEF7EDFC10219B
:1037E0003046FEF76EFD7CBD001401400002300043
:1037F000000C0140FEE7704700F01F0201219140DC
:103800004009800000F1E020C0F88011704700F00E
:103810001F02012191404009800000F1E020C0F822
:103820008011704700F01F02012191404009800083
:1038300000F1E020C0F80011704700F01F020121E4
:1038400091404009800000F1E020C0F8001170476D
:1038500070B50F23C47801780122F4B1144C2468A8
:10386000457804F4E064C4F5E064240AC4F1040675
:10387000E3408478B5401C402C4301F1E021230152
:1038800081F80034007800F01F018A404009800070
:1038900000F1E020C0F8002170BD01F01F0082405F
:1038A0004809800000F1E020C0F8802170BD0000D0
:1038B0000CED00E00249084302490860704700002F
:1038C0000000FA050CED00E02DE9F05F00261D2058
:1038D000FFF792FF6C4CDFF8B4B1A4F1B000A77E03
:1038E00090F83810DFF8A8E1DFF8A8A100258F4292
:1038F0007ED0E776A176626A036B5A434FEA12499B
:103900009BF80820120702D51EF8012000E00A46A5
:1039100094F812C0BCF1010F09D004EB4206B6F9CD
:1039200002C0C4F828C0B6F90460E6620CE043F6B1
:10393000FF7CC4E90A5C90F83DC05FEACC7C01D012
:1039400012B102E0052A00D1012600EB47074FF033
:10395000804CBF893F04B7FBF3F3E361476BBCFBCB
:10396000F7F7276294F813C0BCF1000F06D0BCF142
:10397000010F05D03B4403EBD3735B10636201E09E
:103980003B466762DFF810C14FF6FF7707EA83070F
:10399000ACF808709AF8007090F80A8090F83DC072
:1039A000082F08F003070CF0030C05D067450BD176
:1039B000B8F1000F05D008E0674505D0B8F1000F59
:1039C00003D05B42636200E06562C6B1636A002BAC
:1039D00003D006DD228D05E00AE0304B33F81220DB
:1039E00000E0A28DA4F86020227822F0200222704C
:1039F0009AF80020042A07D0082A05D012E0B4F86B
:103A0000603003EB0902EDE780F8405065629BF8F7
:103A10000800000701D51EF80110204830F81100F9
:103A2000A4F860001E49606A09883E314843B4F832
:103A3000601001EB204006B21D20FFF7F3FE606A24
:103A4000002807D021784FEA81600ADD002804DAD7
:103A5000A08D09E0B4F8600006E0E06AB04208DB3F
:103A60000CE0002802DA208D208208E0A06AB04233
:103A700004DD208241F02000207000E026822575C0
:103A800065752586BDE8F09FF8010020A40200209E
:103A9000B49800081B0700202C0A0020C6980008D4
:103AA0002404004043184FF48042934210DD9042BA
:103AB00002DD104600210BE0914202DD002011469C
:103AC00006E08003B0FBF3F000B2C0F5804109B21C
:103AD00041EA00407047F0B500224FF46A740E25A9
:103AE000C460826205824FF48346082746610783DB
:103AF00043F6FF7C4283A0F81CC040F249234FEA02
:103B00008C3E8360C0E9082ECC608A620D824E61D3
:103B10000F834A83A1F81CC08B60C1E9082EF0BD59
:103B2000002181620949C1600E2101824FF6BF5117
:103B30004161082101834FF44041418343F6FF7105
:103B4000818309070162024941627047638A01006B
:103B500000C0FF0F064941F6A260088005480168D1
:103B6000054A01F4E06111430160BFF34F8FFEE7A6
:103B7000442C01400CED00E00400FA0538B50121A9
:103B80000D2000F0A3F94FF4E060ADF80000182418
:103B90008DF8034003258DF8025069460D48FEF765
:103BA0000BFB4FF46040ADF800008DF803400A4C69
:103BB0008DF8025069462046FEF7FEFAA014ADF8D3
:103BC000000048208DF8030069462046FEF7F4FA0D
:103BD00038BD000000080140000C01402DE9F04113
:103BE0000121CE028CB0304600F070F9DFF86C8114
:103BF000404601F07FFC08A801F0A8FE4FF4586091
:103C0000ADF824000024ADF820402020ADF82200BB
:103C10000125ADF826408DF8285008A9404601F04E
:103C200047FE0021404601F09AFE4FF6FF714046E4
:103C300001F09FFE01220021404601F02BFE0121F0
:103C4000404601F013FC04A801F02BFCADF8106015
:103C5000A802ADF81200ADF81440A220ADF816008D
:103C60002803ADF81800ADF81A40ADF81C4004A9BF
:103C7000404601F005FC6027ADF80070ADF8044047
:103C8000ADF80840ADF80C40ADF80240ADF8064084
:103C9000ADF80A40ADF80E406946404601F0EAFC36
:103CA0006946404601F02CFD6946404601F072FD30
:103CB000ADF8045040F61450ADF80070ADF80600B1
:103CC000ADF80840ADF80C40ADF80250ADF80A4030
:103CD000ADF80E406946404601F0A0FD0121404686
:103CE00001F0E8FB0821404601F004FD3146404662
:103CF00001F046FD0821404601F08AFD314640466C
:103D000001F0BEFD7021404601F0C7FD18208DF87E
:103D10002C008DF82D408DF82E408DF82F500BA8DB
:103D2000FFF796FD0D480C30018841F080010180BD
:103D30000A481430018841F001010180001F04800D
:103D40000121404601F0C0FB8DF82850012140467A
:103D500001F0C4FB0CB0BDE8F0810000002C014074
:103D60007047000070B50189C1EB411101EB4101C1
:103D7000CA0B42810B49104603F066FE09480C3815
:103D8000B0F90C200168B0F90E4001FB02F5436860
:103D9000614303FB145503FB0211AD138913C0E902
:103DA000055170BD380A002040F2134141600821DE
:103DB00081608621C1604FF48041016149424161C7
:103DC00000210162C16270470162704710B501882D
:103DD0004288891A09B20183B1F5005F02DBA1F5BF
:103DE000804104E011F5005F02DC01F580410183B0
:103DF000B0F9182041685143C1618368846A534314
:103E0000C2681B12624303EB2222036A1A44114464
:103E100002628A13426241698A4203DB01698A4273
:103E200000DC11468A1AC0E90A21028E4FF403739E
:103E3000594302EBA13202860B4A1278082A04D1B8
:103E40000A4A936F03EBA1319167B0F93010B1F5D5
:103E5000804F02DDA1F5804103E0002902DA01F57F
:103E60008041018610BD00001B070020680A002069
:103E7000034A516821F440410143516070470000FA
:103E800000100240044A0029516901D0014300E0BA
:103E9000814351617047000000100240044A00292C
:103EA000D16901D0014300E08143D1617047000036
:103EB00000100240044A0029116901D0014300E0CA
:103EC000814311617047000000100240044A00293C
:103ED000916901D0014300E0814391617047000086
:103EE00000100240044A0029D16801D0014300E0DB
:103EF0008143D160704700000010024030B5244972
:103F00004A6812F00C03234A03D0042B01D0082B7B
:103F100026D002604A680F231F4C03EA1212A35CEA
:103F20000268DA4042604B68072505EA1323E35C28
:103F300022FA03F383604B6805EAD323E35CDA409B
:103F4000C2604B68032403F4404104EA933303EB5B
:103F50009161114B1B1F595CB2FBF1F1016130BD46
:103F60004A680E4B1A404B68140103F4803303D5A2
:103F7000C2F38342113202E0022404EB924213B1F5
:103F80004B689B0301D5064B00E0024B5A43C0E748
:103F90000010024000127A000400002000003C08DB
:103FA00000093D002DE9F041274CA615402120468F
:103FB000FEF780F9850080212046FEF77BF945EA6F
:103FC000400531462046FEF775F90543EDB2402124
:103FD0002046FEF76FF9870080212046FEF76AF938
:103FE00047EA400731462046FEF764F90743F8B236
:103FF000A842DBD140212046FEF75CF987008021F2
:104000002046FEF757F947EA400731462046FEF7BB
:1040100051F90743F8B2A842C8D140212046FEF723
:1040200049F9870080212046FEF744F947EA400716
:1040300031462046FEF73EF90743F8B2A842B5D113
:104040002846BDE8F08100000010014010B502686C
:10405000416802FB02F301FB01330D4CA34211D96D
:104060001B0E0E3B0B4C9BB212B234F8133009B24C
:104070005A43594342F38F3241F38F31C0E9022151
:10408000012102E0C0E902210021017410BD0000FD
:10409000E10BBF0E288C00082DE9F05FFB48FC49BE
:1040A00002880B889A1A92B20F2A7CD30988018061
:1040B000F84802468189D2884B0703D48B0701D484
:1040C000CB0702D042F4007201E022F40072C280F9
:1040D0008246080702D45046C90604D5BAF806102D
:1040E00041F0010102E0C18821F00101AAF80610A7
:1040F000E848FDF791FEDFF8A0B3BBF93A10B1F53F
:10410000804F03DA491CABF83A1003E04FF48040CB
:10411000ABF83A00DFF8849341F6CC41E04CD9F893
:104120004800884203DDA06820F01000A060DD494F
:10413000DD4E4FF00008088830B1401E088084F83A
:104140000F8086F800802BE0BAF8060042041BD4EA
:10415000BAF80C10CA0617D4090715D4010613D4EF
:10416000810611D401050FD4410603D5CF49097842
:10417000090609D5410707D4C10505D4010703D4B1
:10418000810401D4C0060BD5C94884F80F80C94901
:1041900086F80080A0F81E80A1F8008080F82A80B0
:1041A000E08FC54A00E0DFE0DFF810E340B1401ED9
:1041B000E087107820F00200107084F80F800AE089
:1041C000107840F0020010703078012805D19EF878
:1041D0000000062801D186F800803078B84D01270C
:1041E0000A2873D2DFE800F0FEC005C0FDFCC072F3
:1041F000FBFADFF8ACA240F62823AAF12C0A40F61D
:10420000CC40BAF81610491C89B2AAF816108C4690
:10421000D9F84410994202DAAAF8168010E0DBF8C7
:104220000C3083420CDBB2F90420B2F5005F07DBEF
:10423000BCF5FA6F04D32B7813B9AAF816802F7047
:10424000A04A12881AB1A04A13885B1C1380E37B32
:10425000092B1FD042F6CC42022B74D0A4F8308137
:10426000EA67AA67B4F8400050B3984840F63A228B
:1042700090F86800012833D0C4F8D88084F8EA8028
:10428000CAF82080B4F9301001F21D50904237D89E
:10429000102336E07D484430FEF7F8F8FDF736FE8F
:1042A000E86A40F391008103A86289488162D9F8E5
:1042B0004410CAF8281041F27C51CAF8181083E261
:1042C00044F62060814202DCA88A01E0D3E1404646
:1042D0002086E86A6863A86A2863A4F8407015E03D
:1042E0007C48C4F8D80084F8EA70B4F9301001F2C0
:1042F0001D53934201D8102300E02023102202E036
:1043000020231022002000F0E1FB20866F48724934
:104310004FF4927390F86800012815D0D9F8440042
:1043200040F2DC52904203DAB5F90A209A4215DBDA
:10433000B4F8402040F6C413521C92B2A4F84020B6
:104340009A420BD212E01AE0D9F8442040F2DC5035
:10435000824209DAB5F90A00984205DA86F8008047
:1043600084F8EA80A1F81A80BDE8F09FDBF80C2001
:10437000002AF9DC42F6E0629042EFDAF4E7B4F8A2
:10438000303140F6B836B3420BD2DFF800C1ACF1A1
:104390001C0C9CF800C05FEACC7C02D15B1CA4F82A
:1043A00030311FFA83FC40F2DC539C4503D9A4F85A
:1043B000306143F26662EA67CAF828108AF807702B
:1043C000464EA4F8408084F8EA80727FE2B1F07F24
:1043D000F0B3208DB4F9301000B204E0F1E0CFE08A
:1043E00014E10FE117E10A23052200F06FFB20869C
:1043F00086F81F8086F81D80B4F930004FF48041A4
:10440000884242DD2186AFE7304E96F86820012AC7
:104410000AD1DBF80C2040F23333DA4204DCA32368
:10442000B4F930101A465EE094F84600022803D131
:1044300096F86D00022818D008B2294901F0FCFC5A
:10444000A4F8E400B4F9E410A06A884202DB00E0BA
:104450008CE0084600B2AAF8140096F84D1041B15D
:104460003623B4F9301005223DE008B21C49B031C2
:10447000E4E7D9F8441044F250629142B4F93010A4
:1044800040F247132EDC36222DE073E06009002055
:1044900024070020540A0020300500204801002095
:1044A000A4020020280700201B070020FC06002093
:1044B000F00800201E000020DA0500201C07002064
:1044C000640000202000002022000020B40C002006
:1044D0009008002034F3FFFFD40900207C0C00205A
:1044E0001A8E0008032200F0F1FA2086B4F91601B2
:1044F000B4F91411884208DA96F84D1011B100F1A0
:1045000002000FE000F108000CE00EDD9AF8042034
:1045100002F10102D2B28AF80420022A07D38AF8F3
:104520000480401EA4F8160101E0A4F81611D5E994
:104530001E01884208DA96F84D1011B100F1020010
:1045400010E000F108000DE00EDD9AF8042002F101
:104550000102D2B28AF80420022AFFF44DAF8AF891
:104560000480401EA86747E7A96745E740F26660F8
:10457000208641E70028BFF601AFA4F83080F3E6BB
:10458000C748D4F8DC10814202D2491CC4F8DC10C0
:10459000E17B082903D1D4F8DC1081420DD386F8E1
:1045A0000080A068C10502D520F0080001E040F0BD
:1045B0000800C4F8DC80A060D6E6BDE8F05F02F039
:1045C00085BCE07B092802D0A4F830803BE1B54DE2
:1045D000E869401CE86102280ADD288D012301B248
:1045E000288B052200B200F071FAC5F81C80A86281
:1045F000AD48298D0180B9F844104180FDF75EFF78
:104600002086B1E6BDE8F05F04F0D0B9A748007895
:1046100009287DD0A8E6A34841F28831A0F8168089
:10462000D9F8440088420ADA2878012807D1A0483E
:1046300085F80080A0F800809E48A0F800809E4980
:104640009E4B0888401C82B29D480A80C82A04D329
:1046500090F800C0BCF1010F19D0B2F57A7F04D3F5
:1046600090F800C0BCF1020F11D0B2F5FA6F02D37E
:104670000278032A0BD0E07BA346801E082874D260
:10468000DFE800F011A4E4F8047374A26CE680F88B
:104690000080A1F80080BAF8061021F40061AAF8A1
:1046A00006101F70E7E7FDF73FFE99F800004C4643
:1046B000400612D58348807804280ED0616C2046CD
:1046C00082290ADA817A94F83D0001F0030100F0B2
:1046D0000300814201D001F0AFFD3078062890D070
:1046E00084F83F80A06C784940F311008203E862AF
:1046F00080108A628103A86274488162FDF706FC1B
:1047000068485D46C771BBF81401ABF8160100E0BC
:1047100099E0606CABF88280B0F5437F12DD4FF416
:104720008040A5F88000A86840F48060A86094F8F4
:1047300038100529AAD140F01000CBF8080080E01D
:10474000307011E64FF48041A5F88010A96821F47B
:104750008061A96040F28A21884204DA207840060C
:1047600001D402F09FFAA86868E08EE0D9F844000E
:10477000B0F5437F07DA9EF80010062903D000BF8A
:104780008EF800807AE05248017821F040010170F3
:10479000FDF7BCFB43F6FE705C46ABF81601FDF777
:1047A000C3FD4C4810F8341F21F001010170474946
:1047B000C4F8DC80C1F828804349C1F8288008216A
:1047C0003170C0F84480CFE50920B9E79AF80600B7
:1047D000C006B6D4D9F844004C46B0F57A7F32DD35
:1047E000FDF7A2FD2078400611D5364880780428D0
:1047F0000DD0606C82280ADAA07A94F83D1000F09F
:10480000030001F00301884201D001F015FD84F896
:104810003F80B4F84800ABF8300001B24FF480405C
:104820005D46814200DD2886FDF770FBA86840F4F4
:104830008060A86094F838100529C4D140F01000B9
:10484000A86002207CE786F800808DE5D9F8440056
:10485000B0F5437F03DA9EF80010062990D1BAF82C
:10486000061021F02001AAF80610FDF75DFD0420D6
:1048700066E7FFE79EF80000062801D0377073E571
:104880000A490920087005205AE70E4880F802807E
:104890008EF8008085F85E80ABF8308064E500001B
:1048A000C0D4010078020020A4090020600200208A
:1048B000220000202000002016000020140000200C
:1048C0001500002050040020C0080020900800209F
:1048D0002A070020680A002030B585B00121042095
:1048E000FFF7F4FA4FF40040ADF8100048208DF8BF
:1048F000130004A91848FDF75FFC01210846FFF7E3
:10490000CDFA40F68C20ADF8040003240020ADF869
:104910000040ADF80200ADF806004FF08045694652
:10492000284600F0C5FF1C208DF80C008DF80D40C6
:104930008DF80E4001208DF80F0003A8FEF788FFC8
:1049400001221146284600F08DFE0121284600F084
:10495000BBFD05B030BD00000008014070470000FD
:104960002DE9F041304CE07800285AD12078002819
:1049700057D0401E10F0FF00207052D14FF49670B7
:10498000208272B6294F45F2AA50A7F87200002083
:10499000FDF79AFA264D13202860FDF7A7FAA8BB69
:1049A0003420E86002202861224E6E61286940F0C0
:1049B00040002861FDF79AFA40BB00211E4A0846D4
:1049C0005FEA255312F800C0BCF1FF0F00D00121AF
:1049D000401C80B29842F5D3C1B9C4E906763926A5
:1049E0000127A06910F8011B10F8012BA061E069F4
:1049F00001EB022102886A612F6120F8021BE0614D
:104A0000FDF774FA10B9761EB6B2EAD20120FDF7AE
:104A10005BFA62B601F064FC0848816821F48041C9
:104A20008160BDE8F081000018070020B40C002070
:104A30000020024000FC000800FC0008A402002046
:104A40001948016841F010010160016821F003017B
:104A50000160016841F00201016014484168416051
:104A600041684160416841F480614160416821F4DE
:104A70007C11416041680E4A11434160016841F078
:104A80008071016001688901FCD5416821F0030152
:104A90004160416841F0020141604168C1F3810118
:104AA0000229FAD1704700000020024000100240A5
:104AB0000000280830B5044C039D6080A180E2808E
:104AC0002381658130BD0000480A00200A448242EB
:104AD00001DA10B27047C91A8142FBDD08B2704793
:104AE0002DE9F0434348DFF81081DFF81091C17FD2
:104AF000457A046801260023414A424880292BD385
:104B000001F01F0158F821100C420146096802D03B
:104B100041F4805101E021F480510160CF0417D4A9
:104B20008F0415D5977AFF0707D0538199F800C0F5
:104B30002CF0020C89F800C00AE090F84670BFB172
:104B40004FF0020C012F18D080F8463080F81AC1BF
:104B50000F0B67F34D310160802D2AD305F01F0143
:104B600058F821100C4201680CD041F004010BE010
:104B700080F8466080F81A31EAE780F846C080F88D
:104B80001A61E5E721F0040101604C070DD44C05E2
:104B90000BD5947AE40708D0538199F8005025F09A
:104BA000020589F80050C0F898308C0864F38A2117
:104BB0000160917AC90717D1134991F8641001294E
:104BC00012D11249496C32290CDC0178490709D508
:104BD0000189090506D4D0F8981047F23054A14253
:104BE00004D95681C0F89830BDE8F083491CC0F85C
:104BF0009810F9E7E0050020F0930008DA0500209E
:104C0000540A0020A4020020B40C00204801002017
:104C100010B5FCF7ADF80F48018821F002010180C2
:104C20000C49183109880C4A928E1144094A3432D1
:104C3000118008490C390A8842F001020A80011DDE
:104C40000A884FF6ED531A400A80018841F012019C
:104C5000018010BD0C04004050040020064801886B
:104C6000491C89B20180B1F57A7F04D34188491C7F
:104C700041800021018070473C0700200F4810B59B
:104C8000016841F00101016041680D4A1140416035
:104C900001680C4A11400160016821F48021016023
:104CA000416821F4FE0141604FF41F018160FFF76C
:104CB000C7FE05494FF00060086010BD00100240BB
:104CC0000000FFF8FFFFF6FE08ED00E02DE9F041DF
:104CD0002F4D28884FF00004000629D5FCF7C8F9AD
:104CE0002C4A2D4807231778C8262C49012F22D09B
:104CF0002B4FB7F806C0BCF1000F3ED0B0F80CC087
:104D00004CF0080CA0F80CC0B0F806C02CF4006CF5
:104D1000A0F806C0886820F004008860FC8013704A
:104D2000CE8700204FF49661401C80B28842FBD3AE
:104D30002C80BDE8F0811B4F97F800C0BCF1010F3B
:104D40000FD0BCF1020F11D0B0F806C04CF4006CCB
:104D5000A0F806C0886840F004008860052038701C
:104D6000DDE7B0F80CC04CF0080C03E0B0F80CC064
:104D70004CF0100CA0F80CC0F0E70B4F3C70C7884B
:104D800047F40067C780886840F004008860C6E781
:104D9000102C01401B070020540A0020A402002010
:104DA000600900201C070020390700207047000020
:104DB0002DE9F0434FF08040018A21F0010101828A
:104DC000AC48007800287CD1AB4FF87B002878D124
:104DD000AA48406C322874DCA9488068DFF8A492A5
:104DE0004104A94DB9F804004FF0000403D4401C5D
:104DF000A9F8040028E1002874D02978012611B10F
:104E0000012912D017E14946B0F5BE7FFAD92E70BC
:104E1000CC718C71EC702C72287A0A18401CC0B2CC
:104E2000147228720F28F7D305E1B9F80220494619
:104E3000824201D9EE7100E0EC7192488A79083023
:104E40000F2A15D2CB79082B0BD2C3F10708EB79C7
:104E500012F800C003FA08F363441354CA79521CD1
:104E6000CA71CA79082A03D18A79521C8A71CC7115
:104E700099F80610C8460F2973D10D21FCF762F886
:104E8000A881010A6970C0B2A87088F8064098F835
:104E900016208A4265D198F81510814261D198F8A0
:104EA0000BC07A49032302227948BCF1000F10D0CD
:104EB000BCF1010F02D0BCF1020F14D080F86A20BF
:104EC00000E0CBE091F800C02CF00C0C0CF1080CC9
:104ED0000FE080F86A6091F800C02CF00C0C0CF127
:104EE000040C06E0A9E080F86A3091F800C04CF0AC
:104EF0000C0C81F800C098F80C10B6EB111F04D10F
:104F000080F86E4087F846400EE0B2EB111F04D1E6
:104F100080F86E6087F8466006E0B3EB111F03D19E
:104F200080F86E2087F846200B0717D001F00F019C
:104F3000012901D0022915D080F86C602C7198F8F5
:104F40000D102A7906FA02F30B406B71082A44D23D
:104F5000DFE802F00B124319242F363D80F86C4035
:104F6000ECE768E080F86C20E8E713B180F8704067
:104F700033E080F8706030E013B180F850602CE0CE
:104F800080F8504029E023B180F8656087F803611C
:104F900023E080F8654087F803411EE023B187F8DD
:104FA000F54080F84D4018E087F8F56080F84D60D6
:104FB00013E013B180F868600FE080F868400CE0FF
:104FC00013B180F8666008E080F8664005E013B130
:104FD00080F8676001E080F86740521CD2B22A7105
:104FE000082AAED398F80E102A4A8B0705D587F801
:104FF000F16080F86460568104E087F8F14080F841
:1050000064405481C90702D080F8294001E080F84B
:10501000296098F8111000F86D1FC2781E48012A07
:105020001ED001B3012921D04FF48051A0F8761091
:105030001A493C200870A9F80240A9F80440B9F8C0
:105040000210491CA9F80210B9F80210B1F5FA7F54
:1050500004D940F2F511A9F802102C70BDE8F083D4
:1050600044F21C71E2E74FF40051DFE741F2555181
:10507000DCE700001B070020A402002048010020FC
:10508000001001409C0C0020B4060020C804002041
:10509000B40C0020540A002030050020180700201E
:1050A0002DE9F05FFDF740F98E4D2888A5F1040643
:1050B000C0070AD0308820F008003080288820F00F
:1050C0000900288001F0EEFDD9E02888DFF8189269
:1050D000DFF81882864C80071AD5B9F8001041F025
:1050E0000101A9F80010B8F80000804914315030CF
:1050F000088028884FF6F95108402880308840F011
:1051000004003080FEF74EFF84F83C00BDE8F09FBD
:105110002888784F4007288871D520F0040028801F
:10512000FEF740FF94F83C108142EFD1308820F028
:1051300004003080FDF7D0FA2078410605D594F8B8
:105140004C1094F83B209142E0D03978400621F091
:105150000201397004D5FEF7DFF997F82F7004E0EB
:1051600094F83C00FDF732F90746DFF880B140F6CD
:105170008C2A0BF1180B062F47D294F83800B8424E
:105180003ED03846FDF7A6F82078C00716D094F830
:105190003A0094F8391000F00302914206D0A17A47
:1051A00000F0010001F00101884215D1FDF7FCF982
:1051B000FBF72AFEFDF724FB384689E0FDF7F4F9FA
:1051C000FBF722FEFDF71CFB3846FDF70DFA2078B1
:1051D00040F00100207099E7288820F0080028801E
:1051E000206B810801EBD000504515D2B8F80010B3
:1051F0000844ABF80000308840F0080003E00DE000
:10520000308820F00800308080E7B9F8001041F0C5
:105210000101A9F80010DFE75046E7E700072888FA
:1052200031D520F008002880308820F00800308038
:10523000FEF7B8FE84F83C00FDF74EFA387820F00F
:10524000020038702078400604D5FEF765F997F81B
:105250002F5004E094F83C00FDF7B8F80546062D01
:1052600008D294F83800A842B5D0FDF79DF9FBF7B5
:10527000CBFD2AE02048C18841F04001C180BDE853
:10528000F05FFDF79DBAC006288825D520F01000F4
:105290002880308820F01000308097F838000C28E3
:1052A00002D2401C87F83800387840F0020038708D
:1052B000FEF732F997F82F50787884F8390094F88F
:1052C0003800A84287D0FDF76FF9FDF799FA284614
:1052D000BDE8F05FFDF788B94EF2BE1108402880A6
:1052E00014E70000100400400004004024040040C3
:1052F0004801002050040020540A00202DE9F04FFE
:10530000514F85B0388820F0010038804E48002683
:10531000103006804D4CDFF838A14FF0010894F8AA
:105320005C0042F63029C10774D072B649488169E1
:1053300041F400718161816941F4806181614FF4C0
:105340000040FEF795FD444D00212846FBF7BAFAD0
:1053500000212846FBF7ACFADFF800B100215846DF
:10536000FBF7A6FA00213E48FCF72AF92846FBF78E
:10537000C5FB5846FBF7C2FB4FF46020CDE902069F
:105380008DF8056000968DF810808DF804806946D0
:105390002846FBF745FC01231A460F212846FBF758
:1053A00090FC01212846FBF783FA00204946401C67
:1053B00080B28842FBD328462E600121FBF7C0FC57
:1053C00028688007FCD524484C30006894F85C10AD
:1053D00021F001012144A1F85000FBF77DFA62B6EB
:1053E000FDF7A6FF47F69061AAF8001094F85C005C
:1053F000401CC0B284F85C000C2822D2124914313F
:10540000A1F80080388840F00100388005B0BDE880
:10541000F08FFFE7134920F00100085A1249088075
:10542000114945F65800083908800F4847F25801DD
:10543000001F01800C4920200C390880AAF8009038
:10544000D4E70320A070E1E70008004050040020EA
:105450002C080040001002400024014000280140B8
:1054600008000240AC8F0008202C01400029018870
:1054700002D041F0800101E021F0800101807047FD
:1054800010B50A884B88CC881A438B8823431A436B
:105490000B891A434B8989891A430A43A0F844208F
:1054A00010BD0021018041808180C1800181418146
:1054B000818170470029818802D041F0010101E01B
:1054C00021F00101818070470029018802D041F05C
:1054D000010101E021F0010101807047002930F84D
:1054E000441F02D041F4004101E0C1F30E010180EC
:1054F000704700004B4910B5884202D10121C41405
:1055000086E0B0F1804F09D0474988420DD1012192
:105510000220FEF7CFFC0021022064E001210846B2
:10552000FEF7C8FC002101205DE04049884206D119
:1055300001210420FEF7BEFC0021042053E03C4979
:10554000884206D101210820FEF7B4FC0021082082
:1055500049E03849884206D101211020FEF7AAFC13
:10556000002110203FE03449884206D1012120204B
:10557000FEF7A0FC0021202035E03049884202D10E
:105580000121441444E02E49884202D10121CC0477
:105590003EE02C49884202D101210C0538E02A491D
:1055A000884202D101214C0532E02849884206D1C7
:1055B00001214020FEF77EFC0021402013E0244919
:1055C000884206D101218020FEF774FC0021802052
:1055D00009E0204988420AD1841501212046FEF7BE
:1055E00069FC00212046BDE81040FEF763BC1A4963
:1055F000884202D101210C040AE01849884202D1F4
:1056000001214C0404E0164988420AD101218C048E
:105610002046FEF767FC2046BDE810400021FEF75B
:1056200061BC10BD002C0140000400400008004097
:10563000000C004000100040001400400034014005
:10564000004C01400050014000540140001800404F
:10565000001C004000200040004001400044014088
:1056600000480140002A828901D00A4300E08A43B1
:105670008281704730B5028C22F001020284028CD4
:105680008388048B22F0020224F073050C882C43DB
:105690000D8915434A882A43114DA8420BD0114D5C
:1056A000A84208D0104DA84205D0104DA84202D003
:1056B0000F4DA8420DD122F008054A8923F440730A
:1056C0002A4322F004058A882A438D891D43CB8909
:1056D0002B4383800483C9888186028430BD000007
:1056E000002C0140003401400040014000440140D2
:1056F00000480140028B22F008020A4302837047EF
:1057000070B5028C22F010020284028C8488038B14
:105710000D8823F4E6464FF6FF7303EA052535436B
:105720000E8922F0200203EA061616434A8803EA8D
:1057300002123243104EB04202D0104EB04215D188
:1057400022F080064A8924F4406403EA02123243BC
:1057500022F040068A8803EA021232438E8903EA65
:1057600086062643CC8903EA840434438480058377
:10577000C9880187028470BD002C014000340140BB
:10578000028B4FF6FF7322F4006203EA01211143FA
:105790000183704770B5028C22F480720284028CFF
:1057A0008488838B0D8823F073031D4322F40073D8
:1057B0000E894FF6FF7202EA06261E434B8802EA64
:1057C00003233343104EB04202D0104EB04215D1E5
:1057D00023F400664B8924F4405402EA0323334344
:1057E00023F480668B8802EA032333438E8902EA1E
:1057F00006162643CC8902EA041434438480858348
:10580000C9888187038470BD002C014000340140A9
:10581000828B22F008020A438283704770B5028CA3
:1058200022F480520284048C8288838B0D8823F4B6
:10583000E6464FF6FF7303EA0525354324F4005688
:105840000C8903EA043434434E8803EA06362643BF
:10585000094CA04202D0094CA04205D122F4804458
:105860008A8903EA8212224382808583C988A0F84C
:105870004010068470BD0000002C0140003401403F
:10588000828B4FF6FF7322F4006203EA0121114379
:1058900081837047018582827047828822F070027E
:1058A000828082880A4382807047A0F84010704747
:1058B00030B502881B4B1C4C98420DD0A0420BD037
:1058C000B0F1804F08D0194DA84205D0184DA8421C
:1058D00002D0184DA84203D122F070054A882A430D
:1058E000154DA84206D0154DA84203D022F44075AC
:1058F000CA882A4302808A8882850A88028598425B
:105900000AD0A04208D00E4A904205D00D4A9042DB
:1059100002D00D4A904201D1097A0186012181828B
:1059200030BD0000002C0140003401400004004064
:1059300000080040000C004000100040001400402F
:105940000040014000440140004801404FF6FF7113
:10595000818000210180C18041800172704700294F
:10596000018802D041F0020101E021F00201018032
:1059700070470029018802D041F0040101E021F0C4
:105980000401018070470000204810B590F82010F5
:10599000026801F01F001E4951F820001D49024213
:1059A000086802D040F4803001E020F480300860C4
:1059B00019484FF0000280794106184824D418494C
:1059C00003880C88E31A9CB201230F2C08D30C889F
:1059D00004808468042C03DD124C2478022C05D04A
:1059E000427F012A06D00988418010BD4377C277E3
:1059F0000A88428042880988891A89B240F21A626C
:105A00009142F2D3C37710BD427710BDE00500206C
:105A1000F0930008A4020020540A00207C0C00200F
:105A2000240700201B0700202DE9F0414D680023CA
:105A30001E240F22854202DD0868BDE8F081D1F8FE
:105A4000F450854202DAD1F8F000F6E701EBC20526
:105A50006D68854201DA134600E01446E2185208E8
:105A60005D1CAA42F2D101EBC20351F832505C68CE
:105A7000844202DAD3E9026701E053E90267001BBE
:105A8000C11789053A1B41EA9021D3178005FAF71F
:105A900049FB721BA0FB024601FB0261D31700FB0E
:105AA0000310810241EA94502844C6E72DE9F04FE3
:105AB000DFF8B8B16A48DFF8AC91DFF8ACA190F834
:105AC0000EC0BBF91A70BBF91C60BBF91850BBF9CA
:105AD0006C10BCF1070F48D2DFE80CF08D041A30CF
:105AE000485E7600D9F800208284DAF80020C2846B
:105AF000828CC38CA7EB820212B2A6EB83034A43CB
:105B00001BB2594342F3CF2241F3CF23D11870E0A7
:105B1000D9F800204284DAF80020C284428CA5EB38
:105B2000820213B2C28C4B43A6EB820212B243F341
:105B3000CF24514341F3CF23E11814E0D9F80020DA
:105B4000C284DAF800204284C28C438CA6EB820225
:105B500012B2A5EB83031CB24A43614342F3CF2345
:105B600041F3CF24191949420AB244E0D9F8002080
:105B70008284DAF800204284828C438CA7EB820274
:105B800012B2A5EB83034A431BB2594342F3CF221F
:105B900041F3CF24111914E0D9F800204284DAF837
:105BA00000208284428C838CA5EB820212B2A7EB88
:105BB00083034A431BB242F3CF24594341F3CF221C
:105BC000A11849420BB216E0D9F80020C284DAF8D5
:105BD00000208284C28C838CA6EB820212B2A7EBD7
:105BE00083031CB24A4342F3CF23614341F3CF22E4
:105BF000991849420CB2BBF91E50594605F21E567F
:105C0000A64201DACE8306E0A5F21E55A54201DDCB
:105C1000CD8300E0CC83B1F9204004F21E559542BB
:105C200001DA0D8406E0A4F21E54944201DD0C84D6
:105C300000E00A84B1F9222002F21E549C4202DAEA
:105C4000ABF8224008E0A2F21E529A4202DDABF805
:105C5000222001E0ABF82230417B8173BDE8F08F58
:105C6000A40200203C2401403C28014030050020D3
:105C70002DE9F04704466448654D002602786348E4
:105C8000022AB0F9301004D0082A7DD0092A7CD02D
:105C9000B6E0C27B022A02D1B0F8402052B1A4F88B
:105CA000421069810423B5F908101A460020FEF756
:105CB0000DFF9CE05749DFF86081496A0F14E780C7
:105CC0008068410216D5B4F9020040F2DA21884218
:105CD00077DD40F26A41884205DD00BF0823B4F950
:105CE00042101A4648E0A0F2DA20FAF796FB0022AA
:105CF0004A4B52E0C0F3C001C0F30020DFF820910E
:105D000081420CD1D8F8440040F2BA41884258DDB3
:105D100040F66A118842E1DCA0F2BA4010E0414846
:105D20000078C00611D5D8F8440041F224318842E9
:105D300047DD41F2D4718842D0DCA0F59850243878
:105D4000FAF76BFB00224B4627E0374890F87010BB
:105D5000012903D090F86F00012832D1B4F9020074
:105D600041F6DC6188422CDD42F2341188420DDDBF
:105D7000B4F9421020231A460020FEF7A7FEA4F82B
:105D80004200002819DB1EE033E037E0A0F5F050B8
:105D9000DC38FAF742FB0022244BFAF7AAFA0E226B
:105DA000FAF716FBFAF770FB00B2C0F580407843B3
:105DB0008013A4F84200002F05DCA4F8426002E042
:105DC000FFE7A4F84270B4F84200194FE880D8F811
:105DD00044107964A7F84C0000F07EFBB7F84E0041
:105DE000688198F80A000028388F00D14042288145
:105DF00006E01048B0F87C00688100E069812E81DF
:105E000084F84060BDE8F0871B070020A402002052
:105E10006400002030050020480100200000794087
:105E200000C09240FC060020B40C002000C082405C
:105E3000F0080020680A00202DE9F041B1F9025075
:105E400000232B241522854203DAB1F90000BDE8B6
:105E5000F081B1F9AE50854202DDB1F9AC00F6E750
:105E600001EB8205B5F90250854201DD134600E0E1
:105E70001446E21852085D1CAA42F1D101EB8205DA
:105E8000B5F90230834206DA35F9026C35F9044C73
:105E900031F9221006E01E4631F92240B5F90630EC
:105EA000B5F90410801B091BC5178911AD0345EA1C
:105EB00090458703A1FB070CCA1702FB07C201FB31
:105EC00005219A1BD317FAF72DF9000A40EA016061
:105ED000001900B2B0F5804FB9DB43F6FF70B6E7AA
:105EE00070B5134C40F224452946204600F03EF898
:105EF00000281BD0204600F0C7F82946204600F0B5
:105F00001DF80C4C00212046FBF75AFB2046FBF7FE
:105F1000D5FBC0F164000849C0B20428087201D959
:105F200000F046F9BDE87040FBF70EBC70BD000004
:105F300000380140580002406C0600200A0A012186
:105F40009140C943018070470029818902D041F402
:105F5000005101E021F4005181817047002A828ABA
:105F600001D00A4300E08A438282704730B501F0D5
:105F70001F0201240025C1F3421304FA02F2012B8F
:105F80000FD0022B0FD0838A4FEA112100881342D1
:105F900004FA01F400EA040001D000B1012528460A
:105FA00030BD8389F0E7038AEEE710B5C1F34213F1
:105FB00001F01F040121A140012B07D0022B07D0C3
:105FC0001430002A026805D00A4304E00C30F8E7D8
:105FD0001030F6E78A43026010BD000030B5044679
:105FE000008A85B00D464CF6FF710840E9880143F0
:105FF0002182A1894EF6F3100140A8882A89104316
:106000006A890A431043A081A08A4FF6FF410840E5
:10601000A9890143A1826846FDF770FF19488442AF
:1060200001D1039800E00298A189090400EBC001A6
:1060300001EB0010296801D5490000E08900B0FBA0
:10604000F1F06422B0FBF2F109010B096FF01805C1
:106050006B4300EB8300A3891D044FF0320306D588
:1060600003EBC000B0FBF2F000F0070005E003EB2B
:106070000010B0FBF2F000F00F000843208105B0E3
:1060800030BD0000003801408088C0F30800704730
:10609000F8B501210920FDF719FF01218803FDF75B
:1060A00015FF10258DF803502020ADF800001A4E82
:1060B00003248DF8024069463046FCF77DF8164906
:1060C0000C31086820F02000086018208DF80300CB
:1060D0004020ADF800008DF8024069463046FCF7DC
:1060E0006BF848208DF803008020ADF80000694669
:1060F0003046FCF761F88DF803502801ADF8000038
:106100008DF8024069463046FCF756F8012104201C
:10611000FCF7A4F8F8BD0000000C014030B585B0D4
:10612000FFF7B6FF00244FF4E1300090ADF80840CF
:106130000C201D4DADF80440ADF80A00ADF8064046
:10614000ADF80C4069462846FFF748FF25208DF83A
:10615000100004208DF811008DF8124001208DF8F8
:10616000130004A8FDF774FB012240F224412846E5
:10617000FFF71BFF01212846FFF7E6FEFBF70EFBAA
:10618000012280212846FFF7E9FE0122402128460E
:10619000FFF7E4FE012202210448FBF7A3FAFBF714
:1061A000FDFA05B030BD0000003801404400024057
:1061B00070B51D4D00242878432834D168784628CE
:1061C00031D1A878502807D0512805D0812803D094
:1061D000892801D0212826D1144E7071E978717276
:1061E000A81C891CFAF7E6FEB072717A2944097975
:1061F0003182884217D106F10E00017841F0020188
:1062000001700B48016841F020010160317A0948B2
:10621000002204E02B5D03552A55641CE4B28C4235
:10622000F8D38078707170BDB00700206C06002034
:106230000C0C0140E60B002070B51D20FDF7E7FABD
:10624000FDF76AF91D20FDF7F8FA154890F82F10B0
:10625000144D0623144C85F8381090F83B1095F82F
:106260003B201143012A04D0022A07D0042A0AD075
:1062700010E0827A8A420DD0007B09E0027D8A42DA
:1062800008D0807D04E0827F8A4203D090F820000D
:10629000884200D12370002085F8400070BD0000C6
:1062A00050040020480100201B0700200B4800215B
:1062B0004180A0F1B0018A898280CB891A44C280D2
:1062C0000B8A1A4402814B8A1A444281898A1144FA
:1062D000818143F6FF71C18170470000F801002001
:1062E000084940F61C72B1F90C00904202DA00F540
:1062F0009F7005E041F2E302904201DDA0F59F703E
:10630000C88170476400002038B51348C16941F066
:106310000401C1611E208DF8000002208DF80100EB
:106320008DF8020001248DF803406846FDF790FACD
:106330000A4984200880094947F690602C3108807A
:106340000020091F0880054914310C80091F0880AE
:10635000081F048038BD0000001002400008004003
:1063600030B420491E4A45788B7A114692F83B405A
:1063700091F83910AC4218D14BB10379994202D04F
:106380004379994201D140791AE0807909E0837913
:10639000994202D0C479A14202D182F82F3011E093
:1063A000407982F82F0030BC7047C578AC42FAD1F2
:1063B0006BB1C379994202D0037A994205D1007A30
:1063C00082F82F0030BCFEF723BC407AE9E7437A1D
:1063D0009942E2D00479A142DFD0007AE1E70000DF
:1063E0005004002048010020FEE700002DE9F0479E
:1063F0000446007F012868D13548E1880288511A97
:1064000089B2072916D30088E080B4F9000044F26D
:10641000DD414843401346F6D96148438013A060EC
:10642000401000B2A0814FF08051B1FBF0F0F9F7BD
:10643000EFFF2061B4F90C6096B1B4F902104DF68B
:10644000B05048430014A082B4F904704DF6B05225
:1064500007FB02F24FEA2245E58204D4024603E03C
:106460000020E08330E0424212B22283002D01DBA3
:106470002B4600E06B421BB2DFF8589063839846CE
:106480004FF4804AB24208DAF9F7B9FF2169F9F707
:106490008CFEF9F7E0FF801304E0002901DA48469A
:1064A00000E05046E083B04509DA2846F9F7A7FF37
:1064B0002169F9F77AFEF9F7CEFF801304E0002F87
:1064C00001DA484600E050462084BDE8F08700002D
:1064D0002407002000C0FFFF10B52248234C01789C
:1064E0002148022905D1C17B022902D1B0F8401010
:1064F00029B1008EA4F84E000020208710BD90F82E
:1065000046101A48B0F8440000B239B31849097867
:10651000C1F3810101291BD002291CD0154900BFFC
:10652000FBF7A2FC1149A4F8400080B2483101F009
:106530008BFAB4F94C00B4F94A2041425143891313
:1065400024F8381FB4F9101048438013E08210BDBE
:106550000849D839E4E707496C39E1E705496C3166
:10656000DEE700001B070020A4020020F008002046
:10657000C8040020248D00080348002180F82A1058
:10658000C183018770470000F008002010B50400A7
:106590000B462D4AC3F1000028D56442002B12DAC5
:1065A000A04207DA214600F027FA32F81000C0F5C1
:1065B000404041E00146204600F01EFA32F810004B
:1065C00000F5004038E0A34208DA2146184600F002
:1065D00013FA32F8100000F540402DE0204600F09C
:1065E0000BFA32F81000C0F5803025E0002B12DAEB
:1065F000A04207DA214600F0FFF932F8100000F55A
:10660000804019E00146204600F0F6F932F810000B
:10661000C0F5004010E0A34208DA2146184600F019
:10662000EBF932F81000C0F5804005E053B1204688
:1066300000F0E2F932F81000B0F5004F01DDA0F5EE
:10664000803010BD002010BDB88F0008404380137B
:10665000494300EBA13000220302002B14DDB3F507
:10666000001F01DC802001E04FF4005093FBF0F1AB
:10667000014401EBD1714910814206D0521CD2B2C3
:106680000846062AF2D300E00021C80000B2704795
:1066900002E008C8121F08C1002AFAD170477047EB
:1066A000002001E001C1121F002AFBD17047000049
:1066B0002DE9F047A44CA54821880288511A89B2D7
:1066C0000F297DD30088A4F13C052080288F08B1D4
:1066D000401E28872B789E4AC3F3810001281DD0D5
:1066E000022820D0D18B98489A4FDFF86C92407ED8
:1066F0000026B1F5926F1DD8142819D37820607642
:10670000F88840F01000F88040F26660A88123F01D
:1067100001002870D67389F8006015E0D08B00EB7B
:106720004000C00302E0D08B8C494843010CDAE7FB
:10673000401C04E0B1F5DB6F06D310B1401E60765B
:1067400002E043F001002870B5F90200B5F91430F9
:106750004143C3EBC303C1F38F31C3F3D10303EB55
:10676000510109B2A9829046D28B4FF08053504319
:10677000B5F91620C0F38F30C2EBC202C2F3D102CA
:1067800002EB500000B2E882AA6A42431213EA62A6
:1067900093FBF2F22A63724A1080A2680A44A26054
:1067A000E1680144E160207C401CC0B220740728ED
:1067B00006D942F3CF002883C9106983E66000E060
:1067C000BFE0A66041F6C8012674884204DD298B2B
:1067D000644AB2FBF1F1E981C117890341EA9041B2
:1067E000800342F69B420023F9F79CFCA88456489C
:1067F0002A78A0F13C005C49B0F90600930700FB41
:1068000001F14FEA2141C2F3810215D5012A07D0D7
:10681000022A0BD04FF2685141430914A18011E0C4
:1068200049F68C4250430014A0801FE04CF618310A
:1068300041430914A18025E0012A0DD0022A17D076
:10684000A0806984494948430014E083FBF72CF990
:1068500047480088C0B143E04AF65C324243121414
:10686000A2804BF62C22504300146884E183EDE7AC
:106870004DF2AC5141430914A1804EF27C41414399
:10688000091469843B49DEE795F8200000BB88F8CD
:106890000F6089F80060B5F91A00A0F50C519F3916
:1068A000B1F56E7F18D8617FF42912D93249E8809A
:1068B0002E4AA1F8460050430014A880A1F84400D5
:1068C000FF2085F8200081F828002C493C20087022
:1068D00006E0491C617703E0607F08B1401E6077E5
:1068E000B5F91A10B4F91E0081420EDDA07E7D2894
:1068F00009D9F88840F00800F8802148017821F093
:10690000020101700EE0401C06E0A0F23D10814241
:1069100008DAA07E10B1401EA07603E0F88820F0CF
:106920000800F880B5F91810606908446061217E9C
:10693000491CC9B221761F2903D94011A883666179
:106940002676BDE8F087000004050020240700201B
:10695000A4020020540A00201B070020303301004D
:10696000080A002074E8260BCC0E010048850100BF
:1069700026070020D0450100B40C00201807002095
:10698000DA050020024941F68B308862704700002A
:10699000C804002070B5164C06252078062825D29C
:1069A000DFE800F003080E141A211248FAF740FB42
:1069B000012016E00F48801DFAF73AFB022010E094
:1069C0000C480C30FAF734FB03200AE00948123077
:1069D000FAF72EFB042004E006481830FAF728FBEB
:1069E0000520207070BDFAF743FB2570257070BD3F
:1069F0001C070020FC8D0008090A05D0B0FBF1F04F
:106A0000FF2800D9FF20704700207047D0E90021FF
:106A1000C368521A5A4301EBA2318160416070474A
:106A2000B0F90020B0F90210B0F90630521A5A43FA
:106A300001EBA231818041807047000030B5494BA5
:106A4000188849490A8A801A85B24848484A0F2D51
:106A5000047801F150001DD31D880D82117A0907B9
:106A600013D5022C01D0434912E0434DB0F9021076
:106A7000B5F90050A94205DC02DA01F1020108E093
:106A8000458007E0A1F1020103E0022C02D13B495D
:106A900009884180B0F840101D88691A89B29C2984
:106AA00049D31988A0F84010916A0023B1F5804FAE
:106AB00031DB3349896CB1F5405F2CDD314940F25F
:106AC0006665B1F91010A94212DD43F69915A94285
:106AD00002DB40F2333108E040F23335A1F2666167
:106AE000694343F2333591FBF5F1A0F8441001E01E
:106AF000A0F844302449B2F806510978C1F3810165
:106B00002DB100BFB0F8441001F21E511CE092F804
:106B10004620022A10D0A0F84430022C01D0A0F860
:106B20004430B0F95C10B0F9443001F114029A42DB
:106B30000DDAA0F85C2030BD012901D00229E1D195
:106B4000B0F8441001F23331A0F84410E5E703F146
:106B50001402914203DD1439A0F85C1030BDA0F896
:106B60005C3030BD24070020140000201B070020EB
:106B7000A4020020C6040020C4040020C004002099
:106B80004801002030050020C80400202DE9FC4108
:106B900001210220FDF782F901211920FDF796F964
:106BA00001213C48FBF75AFB4027ADF80070032455
:106BB0008DF802400420384D8DF8030069462846C0
:106BC000FBF7FAFAE001ADF800008DF802401C2056
:106BD0008DF8030069462846FBF7EEFA4FF4E071A2
:106BE0002846FBF770FBA815ADF800008DF80240B1
:106BF00010208DF8030069462848FBF7DDFA4FF4B2
:106C0000A060FCF757FE1D208DF8040001268DF8CA
:106C1000056000258DF806508DF8076001A8FCF787
:106C200017FE1F498C2008801D494FF6FA702C3141
:106C300008806E20091F0880194814300680184803
:106C400008300780164920310D80154AD020121DCA
:106C50001080134A45F2F300183210800A1F45F2E3
:106C6000500010800E4A4FF6FF7038321080121D0F
:106C70001080121D108041F21B10088000F012F8E5
:106C8000FBF79EFD064810300580001F0480BDE81C
:106C9000FC810000000C1A0000100140000C0140B3
:106CA0000004004070B51D20FCF7A6FD2A4D4021D0
:106CB0002846FBF7FFFA840080212846FBF7FAFA02
:106CC00044EA4004A9152846FBF7F4FA0443E0B26D
:106CD000224C84F83C00FBF779FB0546052805D9D2
:106CE0001F48C18841F04001C18001E084F838505C
:106CF0001C48007A000703D594F838001A490D5C47
:106D00004FF6FA702063E062A06260622062E06188
:106D1000A0611648606300206064A06484F83F00AE
:106D200084F84000FBF700FBA07AFF2811D0022076
:106D300084F83D000E48008820662846FBF7A2FF35
:106D4000207820F001002070BDE870401D20FCF785
:106D500069BD0120ECE7000000100140480100205F
:106D6000540A0020A4020020B4980008DCFF0500AB
:106D7000240400402DE9F0434E484F4902880B8817
:106D80009A1A92B20F2A69D3098801804B49098B5C
:106D9000027D00EB42029180017D491CC9B2017560
:106DA00008295BD3002404752246017D00EB4103D2
:106DB000491CB3F90430C9B202EB630212B2017587
:106DC0000829F2D33E4904753E4B4A8044800E7830
:106DD0009D895FEAC67C40F638694FF0030714D0FE
:106DE000A2F22B5C42F6E858C44520D3A1F1020C74
:106DF00026F00204ACF8002047750C7040F22B54CA
:106E0000A24211DA45F004021EE046F001060E70BF
:106E10004A4507DD45F001029A8126F002020A7018
:106E2000477519E0447517E045F002020CE04A4549
:106E30000CDA8775427D12B1521E42750CE046F0A5
:106E400002020A7025F007029A8105E0B30703D514
:106E5000837D2BB15B1E837540888880BDE8F083FD
:106E600042F6AA239A4222DAB1F904302BB941F250
:106E7000CD05AA4201DA4480EEE7134C920302EBFF
:106E8000843241F67244B2FBF4F214B240F233356C
:106E900002464480AC4200DA5580B2F90240E41A5E
:106EA00004F5A374B4F5237FD6D84380D4E74FF418
:106EB0008043FAE7E80A002024070020A40200200B
:106EC000DA050020540A0020C8F1FFFF2DE9F04147
:106ED0006D4CDFF8B8E14FF0000594F83410C807A6
:106EE00006D094F938104B42002958DD0E4657E081
:106EF000674884F83750A4F84250664A90F8380042
:106F000084F840001586CEF80450CEF80850624E42
:106F100040F26663CEF80C50A4F87C3036F81000CE
:106F20005E4E768830444FF6FF7606EA800024F8FD
:106F3000300B4FF0806044F8040CA3202084608460
:106F40005810A084E38440F699102085580060858D
:106F50004FF48050A08541F23330E08541F2666005
:106F6000208641F69910608641F6CC40A0864FF409
:106F70000050E08642F23330208742F2666060873C
:106F800042F69910A08742F6CC40E08782F89D50E7
:106F900041F00100207184F84450BDE8F0811E46A4
:106FA00094F937004242002801DD074600E0174609
:106FB000F61B012E0BD0002800DB02465FFA82F69A
:106FC00084F8380094F84F00012805D041E00029EA
:106FD00000DA1946CEB2F3E794F939305942002B62
:106FE00001DB184600E0084694F93A20C7B2504247
:106FF000002A01DB944600E08446BC4508DD002AF7
:1070000000DA0246D7B2002B00DA0B46D8B207E00E
:10701000002B00DA0B46DFB2002A00DB1046C0B2BC
:1070200004EB4000B0F9501004EB470030F9502F4A
:1070300011444910018084F84F5084F83E5084F880
:107040003D5084F83C5084F83B5084F83A5084F822
:10705000395004EB46007546B0F9500024F8420F51
:10706000BEF80410C82309B26422FDF72FFD686042
:10707000E968401AA9680844A860B5F900104843B7
:10708000C013E860608788E7680A0020C805002010
:1070900048010020A4020020C698000864000020D7
:1070A000F0B4544890F83410C90776D0524990F89B
:1070B0004030002291F838108B426FD04F4CA0F82E
:1070C00072204F4DE65C04468E4294F9374002D060
:1070D000EE5C8E420FD1641C64B280F83740EB5CEA
:1070E0008B4202D1641C80F8374090F937300F2B67
:1070F0001BDD0F2317E0434DEE5C434D8E4202D063
:10710000EE5C8E4211D1641E64B280F83740EB5CB5
:107110008B4202D1641E80F8374090F937406FF0FF
:107120000E039C4201DA80F83730324B90F83F5022
:10713000393390F83740EC5490F83F305B1CDBB2A9
:1071400080F83F30062B01D380F83F2090F939407A
:1071500090F93B309C420ED190F93D40A3420AD1B8
:1071600090F93A4090F93C309C4204D190F93E406D
:10717000A34200D1012280F84F201F4A80F840101E
:1071800090F937501378214A012D0DDD14465E0722
:10719000A46804D544F0080403E028E015E024F0D6
:1071A0000804946080F83510B5F1FF3F0ADA5B07F8
:1071B000936802D523F0080301E043F008039360CD
:1071C00080F83510F0BCFBF7AFB890F84F100129EC
:1071D0000DD1B0F8721043F60953491C89B2A0F8DA
:1071E0007210994203D9A0F8722080F84F20F0BCA9
:1071F00070470000680A002048010020A898000895
:10720000AE980008BA980008C0980008A4020020B0
:1072100010B5D0E900210369114481FB03318C02D0
:1072200044EA93514260D0E9022382FB0332940284
:1072300044EA93521144816010BD000030B52049EA
:10724000204AB1F86A301088C01A80B20F2836D3AD
:107250001088A1F86A001C4D00204FF000432A5C02
:10726000940903D00124B4EB921F24D1D20622D07A
:10727000164A52F820201268134C123434F8104089
:10728000224201EB000494F9722008D00A2A04DBA0
:107290000A6823FA00F4224308E0521C09E012F1C4
:1072A0000A0F05DC0A6823FA00F4A2430A6002E030
:1072B000521E84F87220401CC0B21128CFD330BDBA
:1072C000E005002024070020BC930008BC940008BF
:1072D0002DE9F00779497A480A8903889A1A92B207
:1072E000082A74D300880881A1F12C0042890AB1D0
:1072F000521E4281734A92F82820802A67D302F0F6
:107300003F020A70C2890AB1521EC281B1F9062039
:10731000902A0CDB8A46FF2A09D08146C0890028C2
:1073200055D1694800230078092805D005E0BDE85B
:10733000F007624800F09EB90823644A92F8EA50C8
:107340000DB143F004036248817AC90701D043F0CC
:107350000203D2F808C05FEA0C5101D543F00103E3
:10736000176800215B4EFC0302D596F8654004B116
:107370008021C4885FEA446801D541F040015FEA9A
:10738000845801D541F020015FEAC47801D041F072
:107390001001007A400701D541F008014E480078FD
:1073A000C00701D041F00401A00601D541F0010160
:1073B0000020012D00D1082096F8705085B992F870
:1073C0004620022A04D0012A05D03AB108E072E032
:1073D00040F0030004E040F0020001E040F0010052
:1073E0007A0701D440F02000CCF3C0020025CCF392
:1073F000002C624502D13A0700D4042596F86F208C
:10740000012A01D145F00105344A0027BC46127813
:107410003E46C2F38102012A04D0022A04D0032A84
:1074200004D004E0022602E0042600E010262C4AE4
:1074300064060ED5214C1C342478240609D5147812
:10744000640606D4274A40F6CC44926D6243140C7D
:1074500005E0B2F8AE2040F699146243940B4FF069
:1074600008088AF80A804FF061088AF80B808AF8C9
:107470000C308AF80D108AF80E008AF80F508AF83E
:107480001070270A4B4083F06901414069408AF837
:10749000117079408AF81240614052468AF813C050
:1074A00071408AF8146051754FF4C871A9F80E1034
:1074B000FF20AAF80600BDE8F0077047E0060020AC
:1074C00024070020E00500201B070020A402002064
:1074D000540A0020B40C002044090020C8040020F5
:1074E00048010020140800205148816941F0FC0146
:1074F00081614FF4A060FCF7DDF9FBF7EFF9FCF7D1
:107500003DFBF9F753FBFCF733F9FDF7E5F9FFF71E
:107510003DFBFCF773F8FFF7C5FBFBF751F9454D51
:1075200045494FF40050A5F816018867FEF7F6FDAF
:1075300000214FF4FA5340F2EE220020401C80B2AA
:107540009842FBD3491C89B29142F6D33B480026AE
:1075500080F87260F9F7C0F9F9F772FEFCF73EFBAC
:10756000F9F734FDFEF7D0FE102235493548F8F71B
:107570000AFE01F00BFA344C354FE08820F0400051
:10758000E0803248017821F020010170FA20F88172
:107590004FF49670E887FFF7F5F92E492E48FCF76F
:1075A0009AFA2E48FCF7BCFA2D48416A88472D48C4
:1075B000416B8847FEF7E0FF2B48FAF771FA2B4939
:1075C0004220C8802A49C8603E71E088E081208955
:1075D000208260896082FAF767FDFAF7C9FCFFF73D
:1075E00067F801F073F9FFF7C5FB00F0FBF9FFF74F
:1075F00025FE01F02FF8FEF7C7F9FAF725FBFBF798
:107600005FFBFFF71BFAFCF747FDFAF781FFFAF77C
:10761000B3FF00F07DF8FFF75BFE1348FAF708F9B7
:1076200000F06CFAFDF79CF9FAF770FACDE700006C
:1076300000100240A4020020640000203005002059
:10764000B40C002020060020540A0020480100202D
:1076500018070020C008002090080020080400201F
:1076600038000020E4000020D4090020400700205A
:107670003C040020F0B523490278B0F9064000230D
:107680001F4E31F81210FF2C18D0B0F904701E4DA7
:10769000BC4231DA00EBE40704F00704BF7AA740EC
:1076A0008478FFB23CB190F801C0ACF1010C6445A4
:1076B0001FDA3C061DD455F822200DE056F8222092
:1076C000116012498A79521CD2B28A71022A02D3FD
:1076D0008370C3808B71F0BD11608178491CC9B281
:1076E000817042789142F6D38370C188491CC18071
:1076F000F0BD56F82220EFE755F822201160F4E79C
:107700009C950008CE93000844950008B40600201C
:10771000F0B561486149B0F86C200B889A1A92B2B2
:107720009C2A7BD30988A0F86C105D495D4F91F8C5
:107730002A1001F0070297F84610022A00D1491ECC
:10774000594C80F83E104FF00203E2884FF00001E0
:10775000550401D5012236E0A489E50601D50622AB
:1077600031E0250701D508222DE0550603D44F4D01
:107770002D78AD0601D5042225E0150501D5072297
:1077800021E0150601D50A221DE0950601D50C223F
:1077900019E0150701D50B2215E0550701D4D505D1
:1077A00001D510220FE0D50601D505220BE06507B3
:1077B00003D4A50701D4E40702D080F86E3007E0B7
:1077C000920403D5032280F86E2001E080F86E1049
:1077D000374A384C92F820E0324A251FD2F808C0C8
:1077E0002D4AB2F87060721C92B2BEF1000F0DD03B
:1077F0002CF4000CC7F808C090F86E70B7B11E2FBB
:107800001AD090F86F200AB325E007E04CF4000688
:10781000BE60A0F870200A2A01D22360F0BD142AAD
:1078200001D22B60F0BDA0F87010F0BD2B60A0F865
:10783000701080F86F10F0BD642E04D2A0F8702094
:10784000322AEED3E9E7A0F87010EAE77F1C80F84F
:107850006F70A0F8701090F86F20012A10D0002AE5
:10786000E9D0B0F87060761CB6B2A0F870601E2E39
:10787000D7D323603C2EDED9521E80F86F20D2E78A
:10788000B0F87020521C92B2A0F870202360C82A71
:10789000D1D980F86F10C6E7E0050020240700204A
:1078A000B40C0020A4020020540A0020480100204B
:1078B000C8040020141C0140F0B54248B0F848103C
:1078C000491C89B2A0F8481002297AD33E49002405
:1078D000A0F848400A783D4B042A57D04FF4804125
:1078E000082A0BD0A0F10C02B2F900208A4200DA7B
:1078F0001146B3F980208A4200DA1146344A92696F
:107900008A4200DA11B2418282881D8AC2EB850266
:10791000304D12B22D78C5F381062A4D42F2316600
:107920007243B5F9765092126A431213C2608668A8
:107930001546C6EBC60642F3D102F60202EBA632AA
:107940008260C66C1644C664B0F850707F1CBFB22B
:10795000A0F85070B7F5806F04D3B6120682A0F875
:107960005040C464891A1C4EC26A724340F2555694
:107970004E4302EB4602466A32444262B3F930306B
:10798000B2EB034F06DD1A04426206E01349B1F977
:107990000410B3E7002A00DA4462C162104990F88B
:1079A0003D2091F838108A420BD080F83D10B0F895
:1079B0004210A0F84410B0F84010A0F84210A0F80F
:1079C0004050F0BD300500201B070020A40200201D
:1079D0004C0C0020C8040020C3F5FFFF680C0020F9
:1079E0004801002015481649B0F85A200B889A1A09
:1079F00092B20F2A20D30988A0F85A10B0F90010CB
:107A000041F6515251438913A0F86C100D494FF4BF
:107A100080420B78A0F10C01022B06D1B1F90030A5
:107A2000934202DA1B1D0B8000E00A800021A0F8BF
:107A3000601020F85C1F4280704700003005002075
:107A4000240700201B0700204FF6FF7202EA800285
:107A500010F4404315480ED0B3F5804F14D0B3F561
:107A6000004F4FEA122216D0C2F5807330F813305F
:107A70005B424B8005E0120A30F812304B80C2F5B1
:107A8000807230F812000FE0120AC2F5807330F8ED
:107A900013304B8005E030F81230C2F580725B4243
:107AA0004B8030F81200404208807047B8910008BF
:107AB000104A518A908AD28A16384639A2F11102A8
:107AC00000D54942002A00DA52421144002800DA67
:107AD00040420844084943F6284300B2B1F9362031
:107AE0005A43921340F2D733584302EBA030C88672
:107AF00070470000A402002030050020F0B5904936
:107B000090480A8903889A1A92B23E2A1ED30088A6
:107B1000088101F138004FF4FA63428A9A4202D296
:107B2000521C428200E04382874A92F82220802A37
:107B30000CD302F03F020A70B1F90620402A06DB9E
:107B4000FF2A04D0C2883AB1521EC280F0BDBDE8FF
:107B5000F0407B48FFF78EBD428A9A42F6D3077801
:107B60004FF0010E3A074FF0FF055BD5847A40F2E3
:107B7000DC52630708D444F004038372C28081F8A6
:107B80000BE081F80AE04CE04378072B05D0032B8B
:107B900003D0052B01D0062B07D1660605D444F08F
:107BA00040038372C280052239E0654A5FEA437C64
:107BB00002F138024FF42076127A0DD55FEAC26CDA
:107BC0000AD45FEA446C07D442F0100202723A060B
:107BD00028D4C680192222E0DF0709D0970707D4EE
:107BE000670605D442F002020272C680042216E043
:107BF0009F0709D5170707D4670605D442F0080286
:107C00000272C68003220AE01B070BD5530709D472
:107C1000630607D442F004020272C6800B22CA72C5
:107C20008A72CD80494AB2F92230B2F91A7003F251
:107C30003D140022A74200DB0276414E444C06F17F
:107C40003806A479B6895FEAC46C06F101064FF4E0
:107C5000C874B6B213D58681B6F57A7F05D9017A94
:107C600021F0800101728281F0BD037A1E06FBD4EF
:107C7000828143F080020272C480112035E09F426D
:107C800016DA037E052B13D28681B6F5487F04D918
:107C90008281027A22F040020272027A5606E3D40E
:107CA0005B1C037642F040020272C48002201CE09A
:107CB000284B1C89C4F3C006C4F3002740F2EE240D
:107CC000BE4216D11E78360713D4427E012ACBD18C
:107CD000428BB2F5167F02D2521C4283F0BD827AEB
:107CE00042F002028272C4800F20C8728872CD8076
:107CF000F0BD93F80D714FF40046012F18D1164FC7
:107D000041F6583C7F6C674512DD83F80CE1134B5C
:107D10001E60C38AA34202D25B1CC382F0BD4FF433
:107D2000FA73C3801C23CB728B72CD80C282F0BDEC
:107D3000C2820A4883F80C21001F0660F0BD0000D3
:107D4000C406002024070020E0050020C80400200D
:107D5000540A0020A4020020480100201408014019
:107D60002DE9F05FFE48FF49DFF8FCA3007E0A1D05
:107D7000131D0128504658D030F85A4F0C804188C6
:107D80001180BAF85E001880F84DF94C49F2CD32F6
:107D9000B5F91E106183B5F9200043F6CC4C01EB18
:107DA000400050430014A083B4F92230B4F920609D
:107DB00000FB03F201FB062242F38F326282B4F928
:107DC000167007FB0CF7BF1340F2333C704302FB05
:107DD0000CF201FB130007EBA232E28240F38F307A
:107DE000A082B4F91810E34FC1EBC10141F3D101F6
:107DF00001EBE000E04E2083786C30603169304662
:107E00008847DE49308948800846FDF731FFDFF8B2
:107E100070B301264FF000099BF8000008280CD031
:107E2000618F2182042864D01AE030F8604F0C8002
:107E300041881180BAF86400A5E7D24890F937105C
:107E4000491C022953D890F8741019B1B4F85A009B
:107E5000208205E0618F2182A4F85A1080F87460B6
:107E6000B4F91410B4F90A00C74AF9F723FBE06229
:107E7000BAF91611884204DDC348E162027C9140E0
:107E80008162BB48DFF804E3503847F2A308027868
:107E90004EF24611AAB3012A59D080F8009000BFD3
:107EA0009BF80000042827D0B74AB4F91210B4F99F
:107EB0000800303AF9F7FEFA42F6F821A06288424B
:107EC00000DBA162B24DA06A2860E06A68602846C3
:107ED000FBF748FFAC4F287C443F01286AD0A06ADA
:107EE0003860AC480178C90768D0406967E0608FA6
:107EF000AEE7686A0014E062B87AE8B3A648A06208
:107F0000E0E7FFE7B5F91E2042448A4209D8B5F9F7
:107F1000202042448A4204D8B5F9222042448A42B1
:107F2000BED9A0F80290B7F8AE204946B2F5C87F96
:107F300001D8467006E0B2F5487F01D8022200E081
:107F4000032242708AF80F108BF8001026E080F8A8
:107F50000090B5F91EC04A46C4448C4509D8B5F90D
:107F600020C0C4448C4504D8B5F9225045448D4204
:107F700096D9B7F8AE1000E019E0B1F5C87F01D886
:107F8000467006E0B1F5487F01D8022100E00321E8
:107F9000417042808AF80F208BF80020BEF806104E
:107FA00041F40061AEF80610F9F7D4FF78E74FF41A
:107FB000AF70A4E768693860A86900E0E06A78609B
:107FC00071484438FCF742F825466949A34635F81C
:107FD000100F3C39FFF738FDDFF89481A8F1500805
:107FE000D8F81410C8F87010B5F91010B868B5F9C1
:107FF000122000FB01F4FB68504303FB124444F3DE
:108000008F3703FB0100AF8740F38F34EC87634D5C
:1080100028466F80AC80FEF7E9F9287F08F1180543
:1080200001282ED0604241104DF6B35047433A1418
:1080300069802A808B18A8F80440A8F80630891AAD
:10804000A8F808108AF80C90B8F904305446002BB0
:1080500000DD2673B8F90600002802DD217B891CAB
:108060002173B8F90820002A02DD217B091D217344
:10807000217B072921D2DFE801F0201C341A301EB1
:1080800032004648B0F9203059424A106A80B0F9AF
:108090001E004DF6B351484300142880A8F8043060
:1080A0001318A8F80630101AA8F80800CAE7667373
:1080B00003E0022100E0032161739BF80010384EB9
:1080C0000129384F617BDA460DD0072947D2DFE816
:1080D00001F046EFEEEDECEBEA000421ECE70521C0
:1080E000EAE70621E8E70729F0D2DFE801F03804E3
:1080F000297DA8E2FD0001461846FBF7D3FC286065
:10810000B5F9020040F68151484381136980B5F901
:10811000000040F681525043801328800A18A2F6CE
:108120008152B8F80E305242C3EB620212B2A8F884
:108130000C20002A01DCA8F80C90B8F80C207DE196
:10814000404201B2504200B2FBF7ACFC2860B5F9E6
:10815000020040F6815148438013688024E012E118
:10816000D4090020342C0140A40200203005002056
:1081700064000020480100203C040020F803002097
:108180001B070020680A0020C0080020540A0020B5
:108190002C0A002044090020A2FEFFFF080A00204C
:1081A0000024014000280140B5F9001040F681523A
:1081B0005143891329804218A2F68152B8F80E3033
:1081C0005242C3EB620212B2A8F80C20002A01DC72
:1081D000A8F80C90B8F80C205EE13046F8F744FDA2
:1081E00001231A460721C3E019461046FBF75AFC43
:1081F0002860B5F9020040F6815148438113698037
:10820000B5F9000040F681525043801328800A18C7
:10821000A2F68152B8F80E305242C3EB620212B29B
:10822000A8F80C20002A01DCA8F80C90B8F80C2063
:10823000A4F85A201144A4F85E10084461E15942A0
:10824000404209B200B2FBF72DFC2860B5F90200EC
:1082500040F68151484380136880B5F9001040F61C
:1082600081525143891329804218A2F68152B8F8ED
:108270000E305242C3EB620212B2A8F80C20002A60
:1082800001DCA8F80C90B8F80C20A4F85A2010448F
:10829000A4F85C00084462E13046F8F7E5FC0123ED
:1082A0001A46052164E093E167E138E109E1D9E08C
:1082B000ACE01146FBF7F6FB2860B5F9020040F68A
:1082C0008151484380136880B5F9001040F681520F
:1082D0005143891329804218A2F68152B8F80E3012
:1082E0005242C3EB620200E00FE012B2A8F80C2089
:1082F000002A01DCA8F80C90B8F80C20A4F85C2047
:108300001044A4F85A00084454E1504201B25842C3
:1083100000B2FBF7C7FB2860B5F9020040F68151B7
:10832000484380136880B5F9001040F681525143EC
:10833000891329804218A2F68152B8F80E305242B1
:10834000C3EB620212B2A8F80C20002A01DCA8F8E4
:108350000C90B8F80C20A4F85C201044A4F85E003F
:10836000084455E13046F8F77FFC01231A46062100
:108370003846F8F779FC01213046F8F7EBFB01218C
:108380003846F8F7E7FBB04EBAF80800554630809B
:10839000BAF80A007080BAF81000B0803046F9F7D9
:1083A00093FAB4F85A00F1880844A4F86000B4F8CD
:1083B0005C0031890844A4F86200B4F85E00718959
:1083C0000844A4F86400317EA048012978D034F82C
:1083D0005A1F018061884180A18881809B49028861
:1083E00008310A8042884A80808888809748896A54
:1083F0000830884795F83E0000287DD0F8F738FE11
:1084000015F83E0F401E2870BDE8F09F0146184643
:10841000FBF748FB2860B5F9020040F6815148435C
:1084200081136980B5F9000040F6815250438013F2
:108430000A18A2F681525242288052081144A4F828
:108440005E20A4F85C100844A4F85A0000213046CD
:10845000F8F780FB00213846F8F77CFB01231A4629
:108460000621BAE6404201B2504200B2FBF71AFBC5
:108470002860B5F9020040F68151484380136880B6
:10848000B5F9001040F68152514389134218A2F603
:108490008152524229805208A4F85E201044A4F868
:1084A0005A000844A4F85C0000213046F8F752FB5B
:1084B00000213846F8F74EFB01231A4605218CE6C9
:1084C000B4E019461046FBF7EDFA2860B5F9020052
:1084D00040F68151484380136880B5F9001040F69A
:1084E0008152514389134218A2F681525242298087
:1084F0005208A4F85A2000E09BE01044A4F85E0063
:108500000844A4F85C0000213046F8F723FB002162
:108510003846F8F71FFB01231A460721BCE65942EB
:10852000404209B200B2FBF7BDFA2860B5F902007B
:1085300040F68151484381136980B5F9000040F647
:108540008152504380130A18A2F6815252425208B7
:1085500028801144A4F85A20A4F85C100844A4F818
:108560005E0000213046F8F7F5FA00213846F8F7AA
:10857000F1FA01231A4606218EE61146FBF792FA1C
:108580002860B5F9020040F68151484381136980A3
:10859000B5F9000040F68152504380130A18A2F644
:1085A00081525242520828801144A4F85C20A4F859
:1085B0005A100844A4F85E0000213046F8F7CAFAC1
:1085C00000213846F8F7C6FA01231A460521C9E604
:1085D000504201B2584200B2FBF764FA2860B5F984
:1085E000020040F68151484381136980B5F90000CB
:1085F00040F68152504380130A18A2F6815252422B
:10860000520828801144A4F85C20A4F85E100844A5
:10861000A4F85A0000213046F8F79CFA00213846A9
:10862000F8F798FA01231A4607219BE634F8601FF1
:10863000CFE607480088A0F5D04168393FF4E4AEA2
:10864000BDE8F05FF9F7D4BBD4090020300000206A
:10865000182C01402DE9F041904C9148B4F85A1083
:108660000288511A89B20F296FD30088A4F85A00E2
:108670008C480088DFF83082C0074FF000054FF0CB
:10868000010741D0874AD4E90C1024321388B1EB9A
:10869000530F02D21288511A08444FF4F3718842E2
:1086A00000D208468149B1FBF0F0616CC1F3510181
:1086B000084406466064F7F7B0FE00227C4BF7F7EB
:1086C00018FE4FF040427B4BF7F713FE0E22F7F7F0
:1086D0007FFEF7F7D9FEA4F8A40094F86500401CCB
:1086E000C0B284F86500082834D36C4898F8462056
:1086F000001F03789A4201D0027045806E4A1378B9
:108700006E4A23B1458021E06564A56458E0D8F83D
:108710009410A1F5FA618E4211DD616D8B1C9E42B1
:1087200005DDB0F902100A290DDA491C06E08E4277
:1087300005DAB0F90210002908DD491E4180B0F9C0
:1087400002000A2802DB177001E0A2E015706665DE
:1087500084F865505A484FF4A5420178C1F381016D
:10876000012949D002294AD044F687712181A4F811
:10877000A020B0F9243089B24B439B13A4F89C305D
:10878000B0F90E0000237043B0FBF1F0A16CC0F310
:10879000D100C1EBC101C90200EB9130A064F01718
:1087A000810341EA9641B003F7F7BCFCB4F8A2108C
:1087B000C1EBC101C902C00800EB9130A4F8A200CE
:1087C000616CA06E0844A06694F86C20521CD2B272
:1087D00084F86C20082A05D3C008A4F86E0084F839
:1087E0006C50A5663748384EC3885A0633D498F87B
:1087F0000F20022A06D02CE043F20451B6E744F2DF
:108800004621B3E7B26840F69916B24221DD94F8EA
:10881000382094F88660B2420CD084F8862094F810
:108820003D2002F00106C2F34002964202D1A4F8B4
:10883000825004E0B4F88220B2F5966F05D2B4F805
:108840008200401CA4F8820005E043F08002C28050
:1088500001E0A4F88250114894F83F30B0300C2B5E
:1088600001D2C57400E0C774174A0F4C41F2482684
:1088700092F83C20B4F8824041F2504C0C2B0AD3C1
:10888000B14208DB012A06D0614502DD002C00D18F
:108890008774BDE8F0818574FBE700004801002083
:1088A0002407002000040040A40200204564BD010C
:1088B00000209C40133B3340F6030020F7030020C8
:1088C000C8040020540A00203005002070B5284C50
:1088D000284821880288511A89B23E2947D3008846
:1088E00020802548808B254D8002286069692846B4
:1088F00088472349A868FDF797F822496060CB882C
:108900005A072ED40022B0F1F05F0FD9E089B0F5FC
:10891000FA7F08D943F00400C8801B48017821F091
:10892000020101701CE0401CE0811AE0B0F1D25F4E
:108930000CD94FF4F031A1EB10308003C910B0FB1B
:10894000F1F0206100280CDA22610AE0B0F1C85F82
:1089500003D94FF48040206103E023F00400C88075
:10896000E281D4E90401884200DB0846A06170BDC1
:108970004C0C002024070020A40200208C060020BC
:10898000B0970008540A0020DA05002005494FF48A
:1089900080404861086188610348C18821F4827180
:1089A000C18070474C0C0020540A00202DE9F04192
:1089B000384C394E394F207841F23331C2074FF0ED
:1089C00000050CD0A28962B394F90700002800DAF0
:1089D0004042C0B2032829D240F2AE702AE0A5700E
:1089E000E5732F4AE571A58192F83830237220F0A3
:1089F0000800A18040F0020020703D867560B560DF
:108A0000F560916C490005D041F68461A18140F088
:108A100010002070C0B240F0010020706574BDE805
:108A2000F081658120F01000207015E0042803D249
:108A300040F6510060810FE0052802D240F69910FF
:108A4000F8E740F6CC42062803D3072801D30828CC
:108A500001D2628100E0618197F89D0098B9B088E9
:108A6000102301B2B4F90A003622FCF72FF8706027
:108A7000F168401AB1680844B060B6F90010484384
:108A8000C013F0603886388E10B10120A070C6E7A0
:108A9000A570C4E7680C0020A4060020A4020020F2
:108AA000480100202DE9F041554C2678F0077CD094
:108AB0005448217A544D90F8380081427BD0534A73
:108AC0002346DFF84CC1575C93F90E2093F9073029
:108AD000874203D01CF80170874213D146F002068A
:108AE0005B1C26705BB2E3711CF80110814201D15E
:108AF0005B1CE37194F90710062901DD0621E17181
:108B0000521C1CE0434F17F801C0434F844503D06B
:108B100017F801C0844513D126F002065B1E2670AB
:108B20005BB2E371795C814201D15B1EE37194F920
:108B300007306FF005018B4200DAE171521EA2731B
:108B4000207294F907108A1C042A02D941F6846223
:108B5000A2812C4A012912780ADD2B4B56079B680B
:108B600002D543F0080301E023F00803AB60607016
:108B7000B1F1FF3F09DA5107A96802D521F00801D8
:108B800001E041F00801A9606070F9F7CDFBA07821
:108B9000012810D121488068A3280CDA94F9070035
:108BA000022803DD0220E07105E01EE06FF0010104
:108BB000884200DAE171A089002630B1401E00042D
:108BC000000CA08101D1E671A673E87B04280CD0CB
:108BD000B5F93010512341220020FBF777FF28869A
:108BE000002802D1E07B10B1A670BDE8F0810C48EE
:108BF00006700C480670207820F001002070F4E721
:108C0000680C002048010020A4020020A898000859
:108C1000AE980008BA980008C098000830050020F7
:108C2000380700201B070020743F713D9B3BED3946
:108C30006238F436A13565343F332A322731333078
:108C40004C2F722EA32DDF2C242C722B000000360B
:108C50001C070038AA0A003AAA0A003CCC0C003EC5
:108C6000CC0C0040380E0042380E0044380E00464E
:108C7000380E0048380E004AC711004CC711004E8C
:108C8000C7110050C7110052C7110054C711005638
:108C9000C7110058C711005AC711005CC711005E08
:108CA000C7110060C7110062C7110064C7110066D8
:108CB000C7110068C711006A0000003622020038A0
:108CC0008E03003AB005003CD207003EF409004094
:108CD000160C0042380E00445B100046C7110048D5
:108CE0003313004A9F14004C9F14004E0B16005083
:108CF00077170052771700547717005677170058E8
:108D00007717005A7717005C7717005E77170060B7
:108D10007717006277170064771700667717006887
:108D20007717006A000000368E0300386606003AA6
:108D30003E09003C160C003EEE0E004011110042B0
:108D40003313004455150046C11600482D18004A3B
:108D50009919004C051B004E711C0050271D005234
:108D6000DD1D0054931E0056491F00580020005A74
:108D7000B520005C6C21005E22220060D8220062D7
:108D80008E23006444240066FA240068B025006A3B
:108D90000000003400000036000000380000003AF7
:108DA0000000003C0000003E0000004000000042C7
:108DB0000000004400000046000000480000004A97
:108DC0000000004C0000004E000000500000005267
:108DD0000000005400000056000000580000005A37
:108DE0000000005C0000005E000000600000006207
:108DF0000000006400000066000000684414585839
:108E00005870111158585870411158584870111421
:108E10004858587014115848587033130056951319
:108E20000054B61300525A140050FD14004EA11500
:108E3000004C4516004A761600486C17004672181A
:108E40000044BA190042741B0040911D003EB4203A
:108E5000003C9F22003AE1220038532300368B2445
:108E60000034812500322B2700302028002E58297D
:108E7000002CB02A002A9B2C0028D22D00267C2F03
:108E800000242631002202330020FD34001E5C370E
:108E9000001CCC3C001A873E0018BE3F0016004064
:108EA000001400400012004000100040000E00407E
:108EB000000C0040000A004000080040000600408E
:108EC000000400400002004000000020007200206A
:108ED00000700020006E0020006C0020006A00205E
:108EE000006800200066002000640020006200206E
:108EF00000600020005E0020005C0020005A00207E
:108F0000005800200056002000540020005200208D
:108F100000500020004E0020004CA320004AA32057
:108F2000004847210046EB210044EB2100428F22FC
:108F300000408F22003E7A24003C7A24003A6626C4
:108F40000038512800343D2A0030702D002CA33009
:108F500000287A34002451380020CC3C001C00400A
:108F6000001800400014004000100040000C0040B9
:108F7000000800400004004000000000010203045B
:108F800005000500010203040104000305020000BE
:108F9000F001000036010000F8000000BA000000F7
:108FA0007C0000007C0000007C00000041141411D3
:108FB00011144411141441110000290052007B00C7
:108FC000A400CC00F5001E01470170019901C20107
:108FD000EA0113023C0265028E02B602DF020803B8
:108FE000300359038203AA03D303FB0324044C0474
:108FF00075049D04C504EE0416053E0567058F053E
:10900000B705DF0507062F0657067F06A706CE061B
:10901000F6061E0746076D079507BC07E4070B0811
:10902000320859088108A808CF08F6081D09440924
:109030006A099109B809DE09050A2B0A520A780A59
:109040009E0AC40AEA0A100B360B5C0B820BA80BB3
:10905000CD0BF30B180C3E0C630C880CAD0CD20C32
:10906000F70C1C0D410D650D8A0DAF0DD30DF70DDD
:109070001C0E400E640E880EAC0ECF0EF30E170FB2
:109080003A0F5E0F810FA40FC70FEA0F0D103010BB
:10909000531075109810BA10DD10FF1021114311F4
:1090A00065118711A911CA11EC110D122E1250125F
:1090B00071129212B312D412F412151336135613FE
:1090C00076139613B713D713F613161436145614D3
:1090D00075149414B414D314F214111530154E15DC
:1090E0006D158C15AA15C815E7150516231641161A
:1090F0005F167C169A16B716D516F2160F172C1790
:10910000491766178317A017BC17D917F517111839
:109110002E184A18661881189D18B918D418F01816
:109120000B19261942195D1978199219AD19C81928
:10913000E219FD19171A311A4C1A661A801A991A6F
:10914000B31ACD1AE61A001B191B331B4C1B651BE7
:109150007E1B971BAF1BC81BE11BF91B121C2A1C93
:10916000421C5A1C721C8A1CA21CBA1CD21CE91C70
:10917000011D181D301D471D5E1D751D8C1DA31D75
:10918000BA1DD01DE71DFD1D141E2A1E401E571EB0
:109190006D1E831E981EAE1EC41EDA1EEF1E051F16
:1091A0001A1F2F1F451F5A1F6F1F841F991FAE1FA5
:1091B000C21FD71FEC1F002000006400C9002D0152
:1091C0009201F7015B02C00224038903ED035204FC
:1091D000B6041A057F05E3054706AB060F077307BC
:1091E000D7073B089F0802096609C9092D0A900A9A
:1091F000F30A560BB90B1C0C7F0CE20C440DA60DA8
:10920000090E6B0ECD0E2F0F900FF20F5310B410EE
:1092100015117611D71138129812F8125813B81385
:1092200018147714D61435159415F3155116B01675
:109230000E176B17C91726188318E0183D199919CE
:10924000F519511AAD1A081B631BBE1B181C731CA1
:10925000CD1C261D801DD91D321E8A1EE31E3B1FFC
:10926000921FEA1F41209820EE2044219A21EF21ED
:1092700045229922EE2242239623E9233C248F247F
:10928000E22434258525D72528267826C8261827C0
:109290006827B72706285428A228EF283D298929BE
:1092A000D629222A6D2AB82A032B4D2B972BE12B86
:1092B0002A2C722CBB2C022D4A2D912DD72D1D2E20
:1092C000632EA82EEC2E302F742FB82FFA2F3D309E
:1092D0007F30C030013141318131C13100323F3204
:1092E0007D32BA32F73234337033AC33E733223461
:1092F0005C349534CE3407353F357735AE35E435BB
:109300001A3650368536B936ED362037533786371C
:10931000B737E937193849387938A838D73805398F
:1093200032395F398B39B739E2390D3A373A603A19
:10933000893AB23ADA3A013B283B4E3B733B983BC1
:10934000BD3BE03B043C263C483C6A3C8B3CAB3C90
:10935000CB3CEA3C093D273D443D613D7D3D993D87
:10936000B43DCE3DE83D013E1A3E323E493E603EB0
:10937000763E8C3EA13EB53EC93EDC3EEF3E013F0F
:10938000123F233F333F433F513F603F6E3F7B3FA0
:10939000873F933F9E3FA93FB33FBC3FC53FCD3F73
:1093A000D53FDC3FE23FE83FED3FF13FF53FF93F7E
:1093B000FB3FFD3FFF3FFF3FFF3F0000E7382C35FD
:1093C000002020EF2037202333202620210000809A
:1093D000020004000800100000020004000804005D
:1093E000000200040008001000200040008004007B
:1093F000000000800000004000000020000000107D
:10940000000000080000000400000002000000014D
:10941000000080000000400000002000000010005C
:10942000000008000000040000000200000001002D
:109430000080000000080140000C0140000C0140C9
:10944000000C0140000C0140000C0140000C0140E8
:10945000000C0140001001400010014000100140CC
:1094600000100140001001400010014000100140B8
:10947000001001400014014004080140040C0140A8
:10948000040C0140040C0140040C0140040C014098
:10949000040C0140040C0140041001400410014080
:1094A0000410014004100140041001400410014068
:1094B0000410014004100140041401400808014058
:1094C000080C0140080C0140080C0140080C014048
:1094D000080C0140080C0140080C01400810014034
:1094E0000810014008100140081001400810014018
:1094F0000810014008100140081001400814014004
:109500000C0801400C0C01400C0C01400C0C0140FB
:109510000C0C01400C0C01400C0C01400C0C0140E7
:109520000C1001400C1001400C1001400C100140C7
:109530000C1001400C1001400C1001400C100140B7
:109540000C14014010080140100C0140100C0140A7
:10955000100C0140100C0140100C0140100C014097
:10956000100C01401010014010100140101001407B
:109570001010014010100140101001401010014067
:109580001010014010140140000000000000000015
:10959000000000000000000000000000140801406E
:1095A000140C0140140C0140140C0140140C014037
:1095B000140C0140140C0140140C01401410014023
:1095C0001410014014100140141001401410014007
:1095D00014100140141001401410014014140140F3
:1095E000000000000000000000000000000000007B
:1095F00000000000FFFFFF0F0FFFFFFFFFF0FFFF66
:10960000FF0FFFFFFFFFF0FF0FFFFFFFFFF0FFFF68
:10961000FF0FFFFFFFF0FFFF0FFFFFFFFFF0FFFF58
:10962000FF0FFFFFFFFFF0FFFFFF0FFFFFFFFFF048
:10963000FFFFFF0FFFF0FFFF0000004040000000B1
:109640000004000000400000000004004000000092
:109650000004000000400000000400004000000082
:109660000004000000400000000004000000400072
:109670000000000400000040000400000000008022
:1096800080000000000800000080000000000800CA
:1096900080000000000800000080000000080000BA
:1096A00080000000000800000080000000000800AA
:1096B000000080000000000800000080000800009A
:1096C0000000002020000000000200000020000038
:1096D0000000020020000000000200000020000046
:1096E0000002000020000000000200000020000036
:1096F0000000020000002000000000020000002026
:109700000002000000000060600000000006000091
:10971000006000000000060060000000000600007D
:10972000006000000006000060000000000600006D
:10973000006000000000060000006000000000065D
:109740000000006000060000008002000400080025
:1097500010000002000400080400000200040008D9
:10976000001000200040008004000000FF7FFFFF89
:10977000FDFFFFFFFBFFFFFFF7FFFFFFEFFFFFFF17
:10978000FFFDFFFFFFFBFFFFFFF7FFFFFBFFFFFFFB
:10979000FFFDFFFFFFFBFFFFFFF7FFFFFFEFFFFFF7
:1097A000FFDFFFFFFFBFFFFFFF7FFFFFFBFFFFFFAD
:1097B0000000401F7A1903000000001E8976030094
:1097C0000000C01C3BDF03000000801BD1570400D9
:1097D0000000401A9FE00400000000199E7B050075
:1097E0000000C017E42C0600000080160DF80600EB
:1097F0000000401593DE07000000001408E6080092
:109800000000C012B1110A000000801101650B00B8
:1098100000004010E6E30C000000000F46940E002C
:109820000000C00D467710000000800CB08F1200C1
:109830000000400BD2DE14000000000A5E63170037
:109840000000C008601A1A000000800726FC1C00F7
:109850000000400600002000000000057A192300E7
:109860000000C003D53926000000800258512900AD
:1098700000004001764F2C000000000046252F001C
:109880000000C0FE2AC63100000080FDA12834007F
:10989000000000FB4B1F3800000080F829053B004A
:1098A000000000F6EFFE3C00010203040500020385
:1098B0000405000103040500010205000102030480
:1098C00004050001020355050010AA1A55250030B1
:1098D000AA3A0000AA0A55150020AA2A5535FF3FCA
:1098E00000990008000000204C070000E406000872
:1098F000FC9900084C070020DC090000A066000865
:1099000045020406082D0102030404054806070861
:1099100009136D2B1B088104211355152A400619C4
:109920000801A713A93D1B08CD041AC90401251776
:10993000020604050103148020FF8BAA0A02019C81
:1099400015AA0A551500085920AA2A5535FF3F07C0
:109950002903010504060203127C1573FFFF04FFAF
:109960008080010129025F6402130A130D6A120844
:109970001201100C05040602030101030705052866
:109980000B010203040206070303040C3D0706044F
:109990000509191F191904310506064BAA1A024BAD
:1099A000381E026910312E40FD3969260211042F3C
:1099B000405F020C26405B262ACD551555151239FD
:1099C00002017F0316D0071AFF01013B0261AA0CB6
:1099D00012080108A8147F993F2340331311720A1B
:1099E0001608DC91220312100A17401C12600A1696
:0C99F000901B014913216A0200080000CE
:020000040800F2
:10FC00004A46545A594D46312D4E3330202020203B
:10FC1000050406020301AA0AAA0AAA0AAA0AAA0A4B
:10FC2000AA0ADE3F00100000FF0131000201664613
:10FC300000400040513800400040004000400101B9
:10FC400000400040FF387B257B257B25FF003333B8
:10FC50000201401F00016626B81E6626FFFFFFFF57
:10FC6000FFFF01010100010000000300000200008D
:04FC70000000AA5591
:04000005080000ED02
:00000001FF
